:020000020000FC
:100000000C94993118951895189518951895189578
:100010001895189518951895189518951895189578
:100020001895189518951895189518951895189568
:100030001895189518951895189518951895189558
:100040001895189518951895189518951895189548
:100050000C940107189518951895189518951895EA
:10006000189518950C94F20A1895189518951895E6
:100070001895189518951895189518951895189518
:100080001895189518951895189518951895189508
:1000900018951895189518951895189518951895F8
:1000A00018951895189518951895189518951895E8
:1000B00018951895189518951895189518951895D8
:1000C00018951895189518951895189518951895C8
:1000D00018951895189518951895189518951895B8
:1000E00018951895189518951895189518951895A8
:1000F0001895189518951895189518951895189598
:100100001895189518951895189518951895189587
:100110001895189518951895189518950C94E50646
:100120001895189518951895189518951895189567
:10013000189518950C9467061895189518951895A4
:100140001895189518951895189518951895189547
:100150001895189518951895189518951895189537
:100160001895189518951895189518951895189527
:100170001895189518951895189518951895189517
:100180001895189518951895189518951895189507
:1001900018951895189518951895189518951895F7
:1001A00018951895189518951895189518951895E7
:1001B00018951895189518951895189518951895D7
:1001C00018951895189518951895189518951895C7
:1001D00018951895189518951895189518951895B7
:1001E00018951895189518951895189518951895A7
:1001F00018951895189518951895189544241FBCAE
:1002000037CB7ABC26B8A2BD41F61CBE6EBA0DBE75
:10021000FC0C633C5C1D633E6EE3A33E5C1D633ED1
:10022000FC0C633C6EBA0DBE41F61CBE26B8A2BDE6
:1002300037CB7ABC44241FBCAA594EBE34D514BE59
:10024000AE16863CF81D473E59298B3EF81D473EA9
:10025000AE16863C34D514BEAA594EBE14BEA1BDFE
:100260006FEDFCBDDC252FBEE9383F3FDC252FBEFE
:100270006FEDFCBD14BEA1BD1F1F1F0000000000DC
:10028000181C1E1E1E1E1E1E1E1E1E1E1E1E1C189E
:1002900000000000001F1F1F0F0F0F0F0F0F07039D
:1002A00003070F0F0F0F0F0F00000000001F1F1F8D
:1002B0001F1F1F00001F1F1F050001040302200550
:1002C00020200420000701040306000701060302A2
:1002D00005060520200405070006030205070004A3
:1002E00003020000012020020507010403020507A4
:1002F0000103030205070704202005070704030381
:10030000050701042020000102040800000000018C
:1003100001010124212A21302136213D214121459D
:1003200021040402010149214D21512100002A2A02
:070330002A2A2A2A2A2A2AA0
:100338000000422611006B1E2A21E5212C225E2294
:10034800A622E12241238723C82320246924DD240F
:100358008425B825F0252D260000832E1100EA2BD0
:100368004E2C612C8B2CAA2CD52C052D192D332D18
:10037800482DBB2DD72DEC2D372E4D2E622E702EED
:100388000000F93010009D2EF52E082F322F4B2F2C
:10039800762FA42FB82FD22FE72F4C3068307D301E
:1003A800C130D730EC300001663763374556370225
:1003B800563711C0360B853601DE360156370156E1
:1003C8003701563702DE3605723601B33601C036BC
:1003D800038E3602C03603BC36FB00EF13E224D18D
:1003E80003E330D000EF13E21FD100EF13E21CD17A
:1003F80003E328D008E913E017D103E323D008E981
:1004080013E012D102E01ED008E913E00DD108E094
:1004180019D008E913E008D101E014D000EF13E285
:1004280003D100EF13E200D106E00CD008E913E095
:10043800FBD00CE007D008E913E0F6D000EF13E298
:10044800F3D008958A93802FE4E4F6E000810F7BCF
:1004580000830EE210E0E8D000916406007F00936C
:100468006406082F02950F7010916406102B1093E4
:100478006406E4E4F6E00081006800830EE210E020
:10048800D3D0E4E4F6E000810F77008306EE10E0B5
:10049800CBD000916406007F009364068F700091B2
:1004A8006406082B00936406E4E4F6E00081006823
:1004B80000830EE210E0B8D0E4E4F6E000810F77A4
:1004C800008306EE10E0B0D0899108958A93802FBA
:1004D800E4E4F6E00081006400830EE210E0A4D0BA
:1004E80000916406007F00936406082F02950F7040
:1004F80010916406102B10936406E4E4F6E0008182
:10050800006800830EE210E08FD0E4E4F6E000819A
:100518000F77008306EE10E087D000916406007F15
:10052800009364068F7000916406082B009364069C
:10053800E4E4F6E00081006800830EE210E074D085
:10054800E4E4F6E000810F77008306EE10E06CD05B
:10055800899108950E941E35C801A0E007C0B0E047
:10056800FC01EA0FFB1F0081B1DFA395B0E0FC019D
:10057800EA0FFB1F0081002311F0A13180F3E4E0B2
:100588000C942F355FDF07EC16E2E4DF08951BECCF
:100598001093520018E010935000E1E5F0E010814C
:1005A80013FFFBCF003221F402EC0093550003C087
:1005B80003EC00935500E0E5F0E000810061008362
:1005C800E1E5F0E0008104FFFBCF08ED04BF04E0A3
:1005D80000934000E0E5F0E000810E7F008308957D
:1005E80001E00093280200E300932902089501E046
:1005F8000093300208E30093310208950DE0009360
:10060800200300E40093210300E00093220300E4A8
:100618000093240300EE0093280300EE00932A03BE
:1006280000EE00932A0308950150104098018901B3
:10063800232BD1F708958A93802F04C008EE1DEF6D
:100648000E94F40B8A95082F802F0023B9F789910F
:1006580008950E941D3580E090E0A0E0B0E04EE0F3
:10066800442E1BC0442D50E0440F551F440F551F06
:10067800FA01ED52F94D0080118022803380442D1B
:1006880050E0440F551F440F551FFA01E952F94D28
:1006980000821182228233824A9441E0441610F784
:1006A800E7EDF6E20083118322833383442423C0D9
:1006B800042D10E0000F111F000F111FF801E45066
:1006C800FE4F4591559165917491042D10E0000FEE
:1006D800111F000F111FF801E952F94D0081118116
:1006E800228133810E94A233AC01BD010E944133B3
:1006F800C801D90143940FE04016D0F28C019D0146
:10070800E5E00C942E350E941D3580E090E0A0E0D5
:10071800B0E04EE0442E1BC0442D50E0440F551F5E
:10072800440F551FFA01E15FF84D008011802280C7
:100738003380442D50E0440F551F440F551FFA01D4
:10074800ED5EF84D00821182228233824A9441E0A4
:10075800441610F7E3E1F7E2008311832283338321
:10076800442423C0042D10E0000F111F000F111F97
:10077800F801E450FE4F4591559165917491042D0F
:1007880010E0000F111F000F111FF801ED5EF84D6A
:1007980000811181228133810E94A233AC01BD0105
:1007A8000E944133C801D90143940FE04016D0F2AA
:1007B8008C019D01E5E00C942E350E941D3580E0EA
:1007C80090E0A0E0B0E048E0442E1BC0442D50E08B
:1007D800440F551F440F551FFA01E55BF84D008083
:1007E800118022803380442D50E0440F551F440F60
:1007F800551FFA01E15BF84D008211822282338293
:100808004A9441E0441610F7EFE4F7E200831183BD
:1008180022833383442423C0042D10E0000F111FCA
:10082800000F111FF801E85CFD4F45915591659146
:100838007491042D10E0000F111F000F111FF80113
:10084800E15BF84D00811181228133810E94A2333E
:10085800AC01BD010E944133C801D901439409E0AC
:100868004016D0F28C019D01E5E00C942E350E94D3
:100878001D3580E090E0A0E0B0E048E0442E1BC0C9
:10088800442D50E0440F551F440F551FFA01E159FC
:10089800F84D0080118022803380442D50E0440FB1
:1008A800551F440F551FFA01ED58F84D008211826B
:1008B800228233824A9441E0441610F7E3E7F7E2D4
:1008C8000083118322833383442423C0042D10E042
:1008D800000F111F000F111FF801E85CFD4F459133
:1008E800559165917491042D10E0000F111F000FB0
:1008F800111FF801ED58F84D0081118122813381D3
:100908000E94A233AC01BD010E944133C801D90144
:10091800439409E04016D0F28C019D01E5E00C9467
:100928002E350E941D3580E090E0A0E0B0E046E062
:10093800442E1BC0442D50E0440F551F440F551F33
:10094800FA01ED56F84D0080118022803380442D45
:1009580050E0440F551F440F551FFA01E956F84D52
:1009680000821182228233824A9441E0441610F7B1
:10097800E7E9F7E20083118322833383442423C009
:10098800042D10E0000F111F000F111FF801E45A89
:10099800FD4F4591559165917491042D10E0000F1C
:1009A800111F000F111FF801E956F84D0081118140
:1009B800228133810E94A233AC01BD010E944133E0
:1009C800C801D901439407E04016D0F28C019D017B
:1009D800E5E00C942E350E941D3580E090E0A0E003
:1009E800B0E046E0442E1BC0442D50E0440F551F94
:1009F800440F551FFA01E155F84D008011802280FF
:100A08003380442D50E0440F551F440F551FFA0101
:100A1800ED54F84D00821182228233824A9441E0DB
:100A2800441610F7E3EBF7E2008311832283338344
:100A3800442423C0042D10E0000F111F000F111FC4
:100A4800F801E45AFD4F4591559165917491042D33
:100A580010E0000F111F000F111FF801ED54F84DA1
:100A680000811181228133810E94A233AC01BD0132
:100A78000E944133C801D901439407E04016D0F2DF
:100A88008C019D01E5E00C942E359A938A93842F6E
:100A9800682F70E0660F771F660F771FFB01E15321
:100AA800F84D008011802280338000191109220935
:100AB8003309052E1124A00160E070E00E94803205
:100AC800482F50E0440F551F440F551FFA01E153BA
:100AD800F84D4081518162817381040F151F261FD3
:100AE800371F90E0880F991F880F991FFC01E15369
:100AF800F84D008311832283338389919991089556
:100B08001091480001E0009348002091A000309126
:100B1800A2000091A2000C7F04600093A2004FB7CE
:100B28007894E8E4F0E00081016000835091CD0101
:100B3800EF93FF930F932F93EBECF1E008ED21E097
:100B480004BF20832F910F91FF91EF9103E0009351
:100B5800CD018895109348002093A0003093A200FF
:100B68005093CD014FBF0895EFECF1E0008107FDF0
:100B7800FBCF0895F9DFEFECF1E0008101FF11C030
:100B880006E30093CA01EF93FF930F932F93EBECC7
:100B9800F1E008ED21E004BF20832F910F91FF9130
:100BA800EF9108959A938A93C801DEDFFC01E05C17
:100BB800F140B89750F440918F2950E009E010E0D7
:100BC8000E94E731800F911F17C0803901E090071C
:100BD80098F440918E2950E00DE110E00E94E73131
:100BE800980140918F2950E007E510E00E94E73115
:100BF800200F311F820F931F082F0093C001892FE8
:100C08008F718093C10100E00093C20106E0009358
:100C1800CA01EF93FF930F932F93EBECF1E008EDEC
:100C280021E004BF20832F910F91FF91EF91009154
:100C3800C4018991999108950E941F35C801A22F76
:100C480000E000930609FC01E05CF140B89750F41D
:100C580040918F2950E009E010E00E94E731800FB1
:100C6800911F17C0803901E0900798F440918E29B0
:100C780050E00DE110E00E94E731980140918F2982
:100C880050E007E510E00E94E731200F311F820F86
:100C9800931F70DF03E30093CA01082F0093C0017C
:100CA800892F8F718093C10100E00093C201A09346
:100CB800C40105E30093CA0123DF03E0009306099A
:100CC800E3E00C9430359A938A93FA93EA930A9264
:100CD8007A936A935A934A933A932A931A930A9364
:100CE8000FB6E0E0F2E000810460008300914E2935
:100CF8000395077000934E2900914E2910E0000FCC
:100D0800111FF801E35DF74D0081118100933A034B
:100D180010933B0300914E2910E0000F111FF801BA
:100D2800E35EF74D00811181009338031093390376
:100D3800009153290023B1F10091BD281091BE28DC
:100D4800212F220F220B322F40914E2950E0440FC1
:100D5800551F440F551FFA01E358F74D4081518143
:100D680062817381400F511F621F731F408351833B
:100D7800628373838091CB289091CC2801968093CD
:100D8800CB289093CC280091CD281091CE2880179D
:100D9800910741F400E00093532910E00093CB2819
:100DA8001093CC280FBE0991199129913991499135
:100DB8005991699179910990E991F991899199915C
:100DC80018954A933A932A931A930A934FB7209106
:100DD80010023091110200917D29102F110F110B73
:100DE800201B310B2093BD283093BE284FBF09919B
:100DF800199129913991499118958A927A926A9212
:100E08005A924A92BA93AA939A938A93FA93EA9334
:100E18003A922A921A920A927A936A935A934A9326
:100E28003A932A931A930A938FB600915329002371
:100E380009F0BBC380914B2990914C29019680936E
:100E48004B2990934C29803707E1900749F400E03B
:100E580010E000934B2910934C2901E000937A2964
:100E6800009172290023E9F0009172290A950093F4
:100E78007229002321F400E00093400912C0009178
:100E8800672910917329019F4091722950E08001D0
:100E98000E94E73143E00E94FB3100936A091093F6
:100EA8006B09009170290B5F00936D29A3E00091F5
:100EB8007029A01B009163290A3031F400916D2933
:100EC800039500936D29AA95AA230AF4A0E000913E
:100ED8007029043019F405E000936D2980E035C0CD
:100EE80050916D29482F642F082F10E0000F111F13
:100EF800000F111FF801E358F74D0081118122817D
:100F080033814A2F0E945532462FBFDD482F50E0CB
:100F1800440F551F440F551FFA01E356F74D008340
:100F280011832283338300E010E020E030E0482F73
:100F380050E0440F551F440F551FFA01E358F74D71
:100F480000831183228333838395883048F20FEF1F
:100F58000093532900E010E020E030E0EDEDF8E2E6
:100F68000083118322833383E9EDF8E20083118340
:100F78002283338300E010E020E030E0EAE8F9E281
:100F8800008311832283338380E095C0082F10E00B
:100F9800000F111F000F111FF801E356F74D408194
:100FA800518162817381082F10E0000F111F000F1B
:100FB800111FF801E356F74D008111812281338119
:100FC8000E942D320E94E232EAE8F9E24081518122
:100FD800628173810E944133EAE8F9E20083118358
:100FE80022833383E9EDF8E2008111812281338184
:100FF8000E94E23228013901082F10E0000F111F6A
:10100800000F111FF801E356F74D0081118122816D
:1010180033810E94E232482F50E0440F551F440F9D
:10102800551FFA01E35CF74D40815181628173815C
:101038000E94A233A201B3010E9441330E94EF3201
:10104800E9EDF8E20083118322833383EDEDF8E2C2
:1010580000811181228133810E94E2322801390105
:10106800082F10E0000F111F000F111FF801E356A1
:10107800F74D00811181228133810E94E232482F8D
:1010880050E0440F551F440F551FFA01E35AF74D1E
:1010980040815181628173810E94A233A201B30110
:1010A8000E9441330E94EF32EDEDF8E20083118394
:1010B800228333838395883008F468CF40E050E07A
:1010C80060E071E4EAE8F9E200811181228133816C
:1010D8000E941B340E949D39EAE8F9E200831183DB
:1010E800228333830091D1281091D22820E030E068
:1010F8000E94ED32A801B901EAE8F9E20081118104
:10110800228133810E941B340E94EF320093C92848
:101118001093CA28BA2FBB0FBB0BFD01EE5DFC4F25
:10112800449150E00091C9281091CA280E940132C8
:101138000093C9281093CA28E9EDF8E200811181CB
:1011480022813381E9EEF8E200831183228333831D
:10115800EDEDF8E20081118122813381EDEEF8E2B4
:10116800008311832283338300915D29002309F0D2
:101178006FC000915F29013011F481E001C085E062
:10118800E5EFF8E20081118122813381E9EEF8E28E
:10119800408151816281738104171507260737073B
:1011A80094F490E0A0E0B0E0E5EFF8E2008111816E
:1011B80022813381080F191F2A1F3B1F00831183C7
:1011C8002283338311C090E0A0E0B0E0E5EFF8E2BD
:1011D8000081118122813381081B190B2A0B3B0BDB
:1011E8000083118322833383E1EFF8E200811181C8
:1011F80022813381EDEEF8E2408151816281738171
:10120800041715072607370794F490E0A0E0B0E02C
:10121800E1EFF8E20081118122813381080F191F63
:101228002A1F3B1F008311832283338311C090E060
:10123800A0E0B0E0E1EFF8E2008111812281338182
:10124800081B190B2A0B3B0B008311832283338362
:10125800009152290023D9F000E000935229E9EEC9
:10126800F8E20081118122813381E5EFF8E2008301
:10127800118322833383EDEEF8E20081118122810C
:101288003381E1EFF8E20083118322833383E5EFB2
:10129800F8E20081118122813381E9EEF8E2408190
:1012A800518162817381401B510B620B730B408328
:1012B800518362837383E1EFF8E200811181228117
:1012C8003381EDEEF8E24081518162817381401BE8
:1012D800510B620B730B4083518362837383E9EE76
:1012E800F8E20081118122813381E1E2F9E2008391
:1012F800118322833383EDEEF8E20081118122818C
:101308003381E5E2F9E2008311832283338300917C
:101318005F29013009F077C000916B29013029F568
:10132800E9EEF8E200811181228133810E94E232E4
:101338000E942D030E94EF32E1E1F9E2008311835C
:1013480022833383EDEEF8E200811181228133811B
:101358000E94E2320E9487030E94EF32E5E1F9E23F
:10136800008311832283338366C000916B29023086
:1013780029F5E9EEF8E200811181228133810E948A
:10138800E2320E94E1030E94EF32E1E1F9E20083D8
:10139800118322833383EDEEF8E2008111812281EB
:1013A80033810E94E2320E943B040E94EF32E5E161
:1013B800F9E200831183228333833DC0E9EEF8E22A
:1013C80000811181228133810E94E2320E949504BA
:1013D8000E94EF32E1E1F9E2008311832283338333
:1013E800EDEEF8E200811181228133810E94E23220
:1013F8000E94EF040E94EF32E5E1F9E200831183D5
:101408002283338318C0E9EEF8E20081118122813A
:101418003381E1E1F9E20083118322833383EDEE26
:10142800F8E20081118122813381E5E1F9E200834C
:10143800118322833383E1E1F9E200811181228162
:101448003381E9E1F9E24081518162817381400F82
:10145800511F621F731F4083518362837383E5E1C9
:10146800F9E20081118122813381EDE1F9E24081C5
:10147800518162817381400F511F621F731F408326
:10148800518362837383E1E2F9E200811181228151
:101498003381E9E2F9E24081518162817381400F31
:1014A800511F621F731F4083518362837383E5E278
:1014B800F9E20081118122813381EDE2F9E2408174
:1014C800518162817381400F511F621F731F4083D6
:1014D80051836283738320917629239520937629FB
:1014E8000091702910E0F801EF5DFC4F049120177E
:1014F80008F45BC000E000937629E9E1F9E2008195
:10150800118122813381E1EEF8E200831183228385
:10151800338300E010E020E030E0E9E1F9E2008305
:10152800118322833383EDE1F9E200811181228165
:101538003381E5EEF8E2008311832283338300E0F0
:1015480010E020E030E0EDE1F9E20083118322832E
:101558003383E9E2F9E20081118122813381E1E3F9
:10156800F9E2008311832283338300E010E020E056
:1015780030E0E9E2F9E20083118322833383EDE26C
:10158800F9E20081118122813381E5E3F9E20083E8
:1015980011832283338300E010E020E030E0EDE2A5
:1015A800F9E200831183228333838FBE0991199155
:1015B8002991399149915991699179910990199095
:1015C80029903990E991F99189919991A991B991C5
:1015D8004990599069907990899018959A938A932F
:1015E800FA93EA933A922A921A920A927A936A930F
:1015F8005A934A933A932A931A930A939FB78091DE
:10160800A0088434E1F401E4D2D00091C128D7D0F5
:101618000091C828D4D0E1EEF8E20081118146E0BB
:101628000E94FB31CCD0E5EEF8E20081118146E062
:101638000E94FB31C4D000917F29C1D0A4C083355A
:1016480061F4009163290A9500936329002309F046
:101658009AC001E00093632996C0843561F4009133
:1016680063290395009363290A3008F48CC009E0C4
:101678000093632988C0863461F400916B2903952F
:1016880000936B29043008F47EC001E000936B29B5
:101698007AC08735F1F40DE48AD087D490D04AE037
:1016A80050E00091C9281091CA280E94013287D0C1
:1016B8000ED485D000916B2982D0009163297FD008
:1016C80000914D2910E0F801EA5FFC4F049177D0B2
:1016D8005AC0853489F409E56AD0009168296FD029
:1016E800F6D36DD000914D296AD000916A2967D050
:1016F8000091702964D047C08E3431F4009164069B
:101708000F73009364063FC08F3431F40091640670
:10171800006C0093640637C000919129063519F4CE
:101728008093672930C000919129093459F4809336
:101738006E2940916E2950E00FEF10E00E94E731CA
:1017480006D121C000919129073439F480934D299D
:1017580000914D290E94CF1316C00091912903349E
:1017680059F480936A29E0916A29F0E03196E09370
:101778002A08F0932B0807C0009191290D3419F419
:101788008093702951D7809391299FBF099119910E
:1017980029913991499159916991799109901990B3
:1017A80029903990E991F991899199911895E1EAEF
:1017B800F8E0108115FFFBCF0093A00808950134CD
:1017C80009F402E40D3409F40EE4093509F408E5D6
:1017D800E1EAF8E0108115FFFBCF0093A008089517
:1017E8009C01C8010197FC01CF01EF2BD9F7169591
:1017F8000795C8010197FC01CF01EF2BD9F7C90163
:1018080008950E941E3500E40E942602AFEF80E092
:1018180002C0A69583958830A8F4BA2F90E005C039
:1018280000E00E946A02B6959395983090F7BB2322
:1018380011F001E001C000E0002391F70FE10E94E0
:101848006A02F1CFE4E00C942F359A938A9300E46E
:101858000E94260280E008C090E0FC01E858FD4F95
:1018680004910E946A0283958034B0F3899199911A
:1018780008950E941E35D80180E090E02AC00DE24C
:1018880010E0AC010E94E731F801EA0FFB1FE836CF
:1018980001E0F00714F0E856F1408F01212F220FE4
:1018A800220B322F0E94E23245E35AEF6EE87CE3C6
:1018B8000E94A2330E94CF38AC01440F551F440F39
:1018C800551FFA01E35CF74D0083118322833383AC
:1018D8000196883000E0900794F2E4E00C942F35EC
:1018E8000E941E35D80180E090E02AC00DE210E089
:1018F800AC010E94E731F801EA0FFB1FE83601E06E
:10190800F00714F0E856F1408F01212F220F220B27
:10191800322F0E94E23245E35AEF6EE87CE30E94E0
:10192800A2330E949531AC01440F551F440F551F37
:10193800FA01E35AF74D008311832283338301961A
:10194800883000E0900794F2E4E00C942F350E9470
:101958001A35D80180E090E013C0FC01E55FFC4F28
:10196800049110E0AD010E94E731000F111F9C01A6
:10197800220F331FF901E35DF74D008311830196B0
:10198800883000E09007C4F500915A29002329F710
:101998008D01212F220F220B322F0E94E2322801C3
:1019A80039018C01212F220F220B322F0E94E232A3
:1019B8004BED5FE069E47FE30E94A2330E94CF38D9
:1019C800A201B3010E94A233280139018D01212F00
:1019D800220F220B322F0E94E232A201B3010E9491
:1019E80041330E94EF329C01220F331FF901E35D5E
:1019F800F74D00831183C3CFE8E00C942B350E9488
:101A080018354801D90180E090E046C00DE210E0A9
:101A1800AC010E94E731A801480D591D483601E084
:101A2800500714F0485651408D01212F220F220BE8
:101A3800322F0E94E232280139018A01212F220F18
:101A4800220B322F0E94E2320801190145E35AEFB6
:101A58006EE87CE3800191010E94A2330E94CF3896
:101A6800A201B3010E94A233280139018D01212F5F
:101A7800220F220B322F0E94E232A201B3010E94F0
:101A880041330E94EF329C01220F331FF901E35EBC
:101A9800F74D008311830196883000E090070CF41D
:101AA800B5CFEAE00C9429350E941E3520E030E0DD
:101AB80000E010E0A4DF66D106E00E941F03E09179
:101AC800C928F091CA28F39708F4D1C080E09CE5B2
:101AD800A1ECB7E400E010E0009396291093972951
:101AE80008C0E6E9F9E2008111810B5F1F4F00830E
:101AF80011830091962910919729083621E0120741
:101B08009CF52091692630916A26009196291091BA
:101B1800972975DF03E00E941F030091C9281091DF
:101B2800CA2820E030E00E94ED32AC01BD010E94DD
:101B3800A434B8F60091C9281091CA2820E030E0F2
:101B48000E94ED32C801D901009196291091972978
:101B58000093922910939329E091C928F091CA28FB
:101B6800B89708F0BECF50C080E09CE5A1ECB7E480
:101B780005E010E0D7D000E010E00093692610934C
:101B88006A2608C0E9E6F6E200811181025E1F4F6D
:101B9800008311830091692610916A26083E27E088
:101BA800120794F52091692630916A2600919229AE
:101BB8001091932924DF03E00E941F030091C92894
:101BC8001091CA2820E030E00E94ED32AC01BD013E
:101BD8000E94A434B8F60091C9281091CA2820E0C0
:101BE80030E00E94ED32C801D901009169261091B8
:101BF8006A260093942910939529E091C928F091B9
:101C0800CA28749708F0BECF20919429309195295D
:101C18000091922910919329F2DE00919429109154
:101C280095290093452910934629009192291091EE
:101C38009329009343291093442930914429232F51
:101C48000EE010E00E942006209143290FE010E0EA
:101C58000E94200630914629232F00E110E00E94BF
:101C680020062091452901E110E00E9420060FEF8F
:101C780000934F29E4E00C942F35309174293130CA
:101C880049F42093732920918029295F220F2093FA
:101C9800722907C030916929329F00926A0910920F
:101CA8006B09009366091093670904E000934009E3
:101CB800089530916829329F00926A0910926B0941
:101CC800009366091093670904E00093400908959A
:101CD8000E941E35D80104E00093400984E090E09A
:101CE8001AC0E0916829F0E031978F01AC010E9499
:101CF800E73100936A0910936B09A0936609B093C2
:101D0800670908EE1DEF6CDD08EE1DEF69DD00E3E5
:101D180015E766DD0197813000E0900714F7E4E0ED
:101D28000C942F352091682930E020936A0930936C
:101D38006B0944E650E00E94E7310093660910936E
:101D4800670904E00093400948E750E00091BF2884
:101D58001091C0280E9419320E5F10917129011B41
:101D68000E941F0300E00093400908958A93812F81
:101D780010E0D8DF00E315E733DD082F10E0D2DFED
:101D88008991089525E531E207EC16E20E9482392F
:101D980000E80E94C60200E310E0C4DF08950E9434
:101DA8002D3140E050E064E672E40E94A2330E94C4
:101DB800EF3208950E941A35C801D9018A019B01A2
:101DC800A801B9012A013B0140E050E060E271E45A
:101DD8000E941B34AC01BD010E944133A201B30132
:101DE8000E942D3140E050E064E672E40E94A23384
:101DF8000E94EF320B3520E0120714F00AE510E0DC
:101E0800063A2FEF120714F406EA1FEFE8E00C94E5
:101E18002B350E941A35D80126E631E207EC16E286
:101E28000E94823900E80E94C602A13000E0B00793
:101E380014F180E0082F10E020E030E00E94ED323D
:101E4800280139018D01212F220F220B322F0E94E8
:101E5800E2320E943835A801B901820193010E943B
:101E6800A43478F5082F07570E9426020EE30E9433
:101E78006A028395DFCF80E008C006E8081B0E944D
:101E880026020CE30E946A028395082F10E020E0E6
:101E980030E00E94ED32280139010FEF1FEFAD014C
:101EA8000E94E731212F220F220B322F0E94E232AB
:101EB8000E943835A801B901820193010E94A43417
:101EC800E0F200E315E78CDCE8E00C942B350E9487
:101ED8001E35A0E0B0E000E00093010204E00E949B
:101EE8001F0380E090E01CC008EE13E079DCE0E01E
:101EF800F2E000810860008300912B020023E1F3E7
:101F080001E000932B020091120210911302A00F1E
:101F1800B11F0091882910918929A01BB10B019646
:101F2800803A00E0900704F300E100930102BB232C
:101F380012F4A0E0B0E044E650E08D010E941932AE
:101F4800E4E00C942F350E941E35A0E0B0E000E0DC
:101F58000093010203E00E941F0380E090E016C096
:101F680008EE13E03DDCE0E0F2E000810860008369
:101F780000912B020023E1F301E000932B02009172
:101F8800120210911302A00FB11F0196843600E0CF
:101F9800900734F300E10093010240E650E08D0120
:101FA8000E941932E4E00C942F35E0E0F2E0008161
:101FB80000610083009133020023E1F301E0009304
:101FC80033024091652950E00091140210911502E6
:101FD8000E9401322091712930E0220F331F220F15
:101FE800331F020F131F08950E941E350EE210E0E2
:101FF80085D4802F0FE210E081D4482F502F8A011A
:10200800212F220F220B322F0E94E23240E0409310
:10201800010241E040930202E0E0F2E040814062C8
:10202800408340913B024423E1F341E040933B026B
:10203800A801B90100E010E02EEA33E40E941B3445
:10204800C801D901009116021091170220E030E072
:102058000E94ED32AC01BD010E94A2330E94EF3212
:102068000C52114020918229322F330F330B020F6B
:10207800131FE4E00C942F3500913F29109140295B
:10208800F8DB00913F29109140292ADC089500913E
:102098003F2910914029EDDB00913F2910914029FB
:1020A8001FDC40916E2950E00FEF10E00E94E731ED
:1020B8004EDC0091BF281091C02800932609109388
:1020C800270908959A938A9301E010E00E94D605A3
:1020D800902F80E002E010E00E94D60510E0802BEF
:1020E800912B8093BF289093C02805E010E00E94B0
:1020F800D605902F80E006E010E00E94D60510E09B
:10210800802B912B80933F299093402907E010E082
:102118000E94D605902F80E008E010E00E94D605C6
:1021280010E0802B912B80934129909342290EE057
:1021380010E00E94D605902F80E00FE010E00E948A
:10214800D60510E0802B912B809343299093442946
:1021580000E110E00E94D605902F80E001E110E038
:102168000E94D60510E0802B912B809345299093EF
:10217800462903E010E00E94D6050093632904E194
:1021880010E00E94D60500934D2909EF11E00E9446
:10219800D6050093642907EF11E00E94D605009345
:1021A8006C290CE010E00E94D60500936E2905EF1B
:1021B80011E00E94D60500936F290CEF11E00E94F0
:1021C800D6050093652902EF11E00E94D605009319
:1021D800742906EF11E00E94D6050093672904EFE1
:1021E80011E00E94D60500935A290DEF11E00E94D4
:1021F800D60500936A290DE010E00E94D6050093E9
:102208006B290AE010E00E94D605802F90E00BE0D1
:1022180010E00E94D605102F00E0802B912B8093B0
:1022280084299093852903E110E00E94D605009344
:10223800702908EF11E00E94D605009358290EEF87
:1022480011E00E94D605009362290AEE11E00E946F
:10225800D6050093822909EE11E00E94D605009365
:102268007C2980E00CC0082F10E000571E4F0E9408
:10227800D60590E0FC01ED5EF74D008383958A302A
:1022880090F3E4E8F9E20081016000838991999173
:1022980008959A938A93902F00915F29002311F44F
:1022A80088E40BC0992312F48CE307C04AE0092F95
:1022B8000E94D73116E0019F802D00E80E94260277
:1022C800082F10E0F801E854FD4F04910E946A02BB
:1022D80001E80E942602082F10E0F801E754FD4F9C
:1022E80004910E946A0202E80E942602082F10E068
:1022F800F801E654FD4F04910E946A0200EC0E9426
:102308002602082F10E0F801E554FD4F04910E94C1
:102318006A0201EC0E942602082F10E0F801E4543A
:10232800FD4F04910E946A0202EC0E942602082FC7
:1023380010E0F801E354FD4F04910E946A020091F5
:102348006F29013009F059C000915F29002311F469
:1023580088E40BC0992312F482E407C04AE0092FED
:102368000E94D73106E0409F802D03E80E94260294
:1023780090E0FC01E854FD4F04910E946A0204E8D1
:102388000E94260290E0FC01E754FD4F04910E9450
:102398006A0205E80E94260290E0FC01E654FD4F1F
:1023A80004910E946A0203EC0E94260290E0FC015C
:1023B800E554FD4F04910E946A0204EC0E94260233
:1023C80090E0FC01E454FD4F04910E946A0205EC80
:1023D8000E94260290E0FC01E354FD4F04910E9404
:1023E8006A0206E80E94260200E20E946A0206ECDF
:1023F8000E94260200E20E946A028991999108953A
:102408000E941E3500916329083010F082E001C057
:1024180081E0E4E8F9E2018107FF02C005E501C0B7
:1024280008E51091C12811230AF48CC02091C12815
:10243800322F330F330B10E0201731070CF082C016
:102448004AE00091C1280E94D731402F4A5F00918D
:102458008429109185290E94FB310170002309F01D
:1024680071C000916C29013031F42091562900E7A0
:1024780017E103DCB2C000916C290230D1F400915D
:10248800C128053134F42091562900EB16E3F5DB19
:10249800A4C00091C1280B3434F0209156290CEACD
:1024A8001DE0EBDB9AC02091562900E717E1E5DB38
:1024B80094C000916C290330C1F420915629A22FB1
:1024C8008BE090E00091C128102F110F110B4AE00A
:1024D80050E00E941932801B910B04E115E0AC0119
:1024E8000E94E7312A2FC9DB78C000916C2904309B
:1024F80089F4209156290EE610E04091C128542F06
:10250800550F550B041B150B42E850E00E94E731AC
:10251800B4DB63C020915629822F0091C128102F67
:10252800110F110B4AE050E00E941932F801ED5EDC
:10253800F74D418150E006E910E00E94E731282F6D
:102548009CDB4BC00091C12800230AF046C0A09133
:102558007E29BA2FBB0FBB0B482F50E000914929A9
:1025680010914A290E941932A017B107B4F584E0E6
:102578004CEE0091C1280E94D731801B482F009152
:102588008429109185290E94FB310170002329F5C7
:1025980042E0009156290E94C931009356290091C2
:1025A8006C29053059F4209156294091132850E0A0
:1025B80006E910E00E94E73160DB0FC00091C128F6
:1025C8000C3E34F02091562900E01DE756DB05C08B
:1025D8002091562908EC1FEA50DBE4E00C942F35D3
:1025E8008A930CE00093672927E731E207EC16E2AB
:1025F8000E94823900E80E94C60200EC0E94C602CE
:1026080011C028E0482F50E008EC10E00E94E731A4
:1026180050DB00E315E7E4D88A95823090F700ECA8
:102628000093670680E2F9CF0E941E358091BF288B
:102638009091C0280196AC01652F660F660B762F26
:1026480000E01CE62CED32E00E94803248E050E0C9
:1026580060E070E00E948032C801D90148EE53E082
:1026680060E070E08C019D010E9480320850009368
:102678007829853700E4900700E0A00700E0B0075C
:1026880024F001E00093712903C000E00093712950
:10269800AED108E010E020E030E0AC01BD010E94BE
:1026A8002D3240E750E060E070E00E9480320093F5
:1026B800CF281093D02845E00091CF281091D0283A
:1026C8000E94F53140E250E00E94E7310093CF28A4
:1026D8001093D0284AE750E00091CF281091D028D5
:1026E8000E9401320093D1281093D2280091CF285C
:1026F8001091D0280093CD281093CE2846E150E0C1
:102708000091712910E0401B510B0091BF281091D6
:10271800C0280E9419320093D3281093D42800911E
:102728007029043021F400E00093772905C0009156
:1027380070290A9500937729E4E00C942F358A9341
:1027480000916229002329F100915D29002309F5F0
:102758002CDC2091622930E002171307D4F480E0C2
:1027680016C028E831E207EC16E20E94823900E838
:102778000E94C60208E710E0D5DA08EE1DEF30D84F
:1027880001E00E94260202E00E941F038395853023
:1027980040F38991089510912002137E109320022E
:1027A8000A95000F000F10912002102B10932002A1
:1027B80002E00E941F0301E000935229089582DC81
:1027C80000916729009368292FDF0E94F101009189
:1027D8005D29002331F400916F29023011F035D8BA
:1027E80002C00E94050C209145293091462900918C
:1027F80043291091442903D94ADC00914D29CBDFA4
:1028080008959A938A93F89410E500E3AFDAD7DF36
:1028180001E00E94260200E117E20E94F40B809179
:10282800BF289091C0280196AC01652F660F660BF2
:10283800762F00E01CE62CED32E00E94803248E062
:1028480050E060E070E00E948032C8019A938A9359
:1028580029E931E207EC16E20E948239229600E863
:102868000E94C60204EC0E94260280E090E008C0A4
:102878008C0100541E4F0E94D6050E946A020196E0
:10288800893000E09007A4F3789401E000935F2971
:1028980000E00093C22801E010E00093862910931D
:1028A800872901E00093522904EB009361290093E2
:1028B800602900E010E020E030E0EDE0F9E200837C
:1028C800118322833383E1E0F9E2008311832283B9
:1028D80033830091D328102F02E0109F002D0E940F
:1028E8001F0301E00E94260200E117E20E94F40B98
:1028F80001E00093542989919991089522E0209349
:10290800CA01F801049000E00093CA01002D08955F
:102918009A938A9390E088E005C0082F10E0EEDFD4
:10292800900F83958631C8F3992309F493E0092F12
:102938008991999108959A938A930BEE11E00E94D8
:10294800D6050F3F99F50CEE11E00E94D6050F3F12
:1029580069F580914B2900917D29800F90E003C093
:102968000E941C3893959817D8F30E941C38802F22
:10297800853008F489E5282F0BEE11E00E94200627
:10298800C7DF202F0CEE11E00E94200620E00DEE9C
:1029980011E00E94200620E00EEE11E00E942006C1
:1029A80000E010E00093D7281093D82889919991D6
:1029B80008959C01A801CA01892F90E04F7F5070AB
:1029C8008C010E94E731080F191FC801840F951F59
:1029D8000796982F80E00FEF10E0041B150BA80155
:1029E8004F7F5070842B952B8C01C901089500EB03
:1029F8000093010202E20093020203E00093040242
:102A080000917129013021F402E00093040203C00F
:102A180003E00093040203E00093200208E200931D
:102A28002102E0E0F2E00081016000830895009156
:102A38006429002349F0009164060F73009364062B
:102A48000AE200933D2908C000916406006C0093D7
:102A5800640600E200933D2900917C29007F002351
:102A680031F400918406037F0093840608C0009126
:102A780084060C60009384060EE200933D290091C1
:102A88007C290F70002331F4E4E4F6E000810E7F26
:102A9800008308C0E4E4F6E00081016000830CE2F2
:102AA80000933D2900917C290F3F19F40BE3009313
:102AB8003D2908950E941435F89400E30E94CB0242
:102AC800009180060C6000938006009160060F60FC
:102AD8000093600600914006006C00934006E0E613
:102AE800F6E0008100620083E0E4F6E00081026025
:102AF8000083E0E4F6E00081016000830091600655
:102B0800006C0093600608E10093110608E1009349
:102B1800120608E10093130608E10093300608E165
:102B28000093540608E1009355060E94F10100EF56
:102B380011E00E94D6050F3F11F481E001C080E04A
:102B480001EF11E00E94D6050F3F11F401E001C02A
:102B580000E08023882351F020E000EF11E00E947C
:102B6800200620E001EF11E00E9420060AEF11E0A4
:102B78000E94D6050F3F11F401E001C000E0E8E033
:102B8800F6E0108111FD0CC0E8E0F6E0108112FDBE
:102B980007C0E8E2F6E02081217011E0212701C09A
:102BA80020E0022B002309F4D4C02AEA31E207EC22
:102BB80016E20E94823900EC0E94C602789402E371
:102BC8000E941F03F89400E000938F2905C000912C
:102BD8008F29039500938F2900918F29043008F0DD
:102BE800B3C000E000938E2913C0B0E0FD01E25DA0
:102BF800FC4F24910A2F10E000541E4F0E9420061B
:102C0800A395A93090F300918E29039500938E29FE
:102C180000918E290330D8F622E001E010E00E94EE
:102C2800200627E502E010E00E94200620E005E0EB
:102C380010E00E94200624EB06E010E00E94200627
:102C480020E007E010E00E94200620EB08E010E0FA
:102C58000E94200620E00EE010E00E94200620E0FE
:102C68000FE010E00E94200620E000E110E00E9442
:102C7800200620E001E110E00E94200626E003E0A3
:102C880010E00E94200622E004E110E00E942006E5
:102C980020E009EF11E00E94200624E00CE010E09B
:102CA8000E94200621E00DE010E00E94200621E0AD
:102CB80007EF11E00E94200621E00AE010E00E94E0
:102CC800200620E80BE010E00E9420062FE20CEF1F
:102CD80011E00E94200620E004EF11E00E94200687
:102CE80025E006EF11E00E94200625E00DEF11E037
:102CF8000E94200621E00EEF11E00E94200620E04D
:102D080002EF11E00E94200621E003E110E00E949A
:102D1800200621E008EF11E00E94200620E005EFE0
:102D280011E00E94200620E00AEE11E00E94200631
:102D380020E20EEF11E00E94200620E009EE11E0EB
:102D48000E942006A0E05DCF20E00AEF11E00E947B
:102D580020060AEF11E00E94D60500938F29009102
:102D6800480600730093902900919029003321F4BC
:102D780000E000938E290FC000919029003221F4C1
:102D880001E000938E2907C000919029003119F4C1
:102D980002E000938E2913DD03E20093010807E0A7
:102DA8000093000806E910E000932608109327080E
:102DB80080916A2990E0019680932A0890932B08C5
:102DC80000916A29002331F400E010E000932608FE
:102DD8001093270801E0009300090091BF28109183
:102DE800C028009326091093270903E000930609D9
:102DF8000091A20007600093A20007E0009340083A
:102E080004ED11E0009366081093670801E0009351
:102E180046080E94020300919300043019F400E16F
:102E28000093220304DE00917C290F70002309F12E
:102E3800E1E4F6E000810860008303E00093A50860
:102E480009E60093A60802ED0093A70808E100939D
:102E5800A40800E10093A308E2EAF0E00081016021
:102E6800008300E0009368290093692900E000933B
:102E78009129BDDD00E210E041DD00930C0201E282
:102E880010E03CDD00930D0202E0009322020E9454
:102E9800FB020E94F40200914D297DDCF8D80091D4
:102EA8006329002321F400E010E00E94AB0C03E248
:102EB80000934109009164060F7300936406E8E0EB
:102EC800F6E0008103FF8CDB80918F2990E001966A
:102ED8009A938A932CEB31E207EC16E20E9482392E
:102EE800229600EC0E94C60207EC0E942602A0E08F
:102EF80009C00A2F10E000541E4F0E94D6050E94F8
:102F08006A02A395A930A8F30091930010E01A93E0
:102F18000A9325EC31E207EC16E20E9482392296E8
:102F280000E80E94C60200ED17E00E946C0E00EA5D
:102F38001FE00E946C0E00E41FE10E946C0E08EE78
:102F48001DEF0E94F40B00ED17E00E946C0E00E0EC
:102F5800009340090091D328102F02E0109F002D04
:102F68000E941F030091C7260B3409F0A0CF0091DF
:102F7800C826003509F09BCF0091C9260F3409F007
:102F880096CF00916429002331F0009164060F73F5
:102F98000093640605C000916406006C0093640603
:102FA8000091CA26043509F082CF02E000937B29FC
:102FB8000BEE11E00E94D605902F80E00CEE11E098
:102FC8000E94D60510E0802B912B8093D5289093F2
:102FD800D6280DEE11E00E94D605902F80E00EEE67
:102FE80011E00E94D60510E0802B912B8093D72802
:102FF8009093D8280091D5281091D628DADC209112
:10300800D7283091D82802171307A1F481DC402F64
:1030180050E02FEF30E00091D7281091D8280F7F8B
:103028001070201B310B4217530721F402E0009364
:103038007B2950C001EF11E00E94D6050430A8F5A5
:1030480001E000937B2927ED31E207EC16E20E94AC
:10305800823900E80E94C60200EF11E00E94D605FE
:10306800802F01EF11E00E94D605202F0CE310E01D
:1030780090E0081B190B1A930A9303E010E030E064
:10308800021B130B1A930A9329EE31E207EC16E29E
:103098000E948239249600EC0E94C60208EC0E9425
:1030A8001F0304E60E941F0315C000E000937B295C
:1030B80001E00093542900E0009379290CE0009383
:1030C80050290FEF00935D2906E000935B2900E08B
:1030D8000093A4080E94A70F0093882910938929B8
:1030E80008EE1DEF0E94F40B00E000937D29A0E09C
:1030F80016C0E0E0F2E00081046000830091230242
:103108000023E1F301E000932302009110021091E3
:10311800110210917D29100F10937D29A395AA30D3
:1031280040F34AE000917D290E94D73100937D2920
:1031380078940CE00E94260208EE1DEF0E94F40B22
:10314800FEDAE8E0F6E0008101FD24C0E8E0F6E000
:10315800008102FD1FC00FEF00935D2901E000937D
:103168005B2901E000935E2901E00E94260210E538
:1031780000E30E94BA0E2EEF31E207EC16E20E943D
:10318800823900E80E94C602E8E0F6E0008102FF0A
:10319800FBCFD8C0E8E0F6E0008102FD21C00FEFC8
:1031A80000935D2907E000935B2902E000935E2904
:1031B80001E00E94260210E500E30E94BA0E2FE00B
:1031C80032E207EC16E20E94823900E80E94C60249
:1031D800E8E0F6E0008102FFFBCF0E94050CB2C0D8
:1031E80000E000935E290AE00E941F030E946B0F13
:1031F8003801A091D32858C04091BF285091C028C9
:103208004F5F5F4F652F660F660B762F00E01CE659
:103218002CED32E00E94803248E050E060E070E03F
:103228000E948032C8017A926A929A938A9329E41A
:1032380032E207EC16E20E948239249600E80E94E6
:10324800C6020091C9281091CA281A930A9329E541
:1032580032E207EC16E20E948239229600EC0E94C4
:10326800C6020091702910E0000F111FF801EF5EEF
:10327800FC4F059114911A930A9300914D2910E07F
:10328800F801EA5FFC4F049110E01A930A9325E6CF
:1032980032E207EC16E20E948239249608EC0E947A
:1032A800C60204E00E941F030A2FA02FAA9500233C
:1032B80009F0ADC001E00E94260200E21EE40E946F
:1032C800F40B00917D29033344F410E000917D292B
:1032D8000E3C1CF010601123C1F02CE632E207EC22
:1032E80016E20E94823900E80E94C60200ED10E052
:1032F8000E94960E00EB10E00E94960E00ED10E082
:103308000E94960E04E10E941F0305E0601600E08B
:103318007006C4F429E732E207EC16E20E9482390B
:1033280000E80E94C60200ED10E00E94960E00EB35
:1033380010E00E94960E00ED10E00E94960E04E147
:103348000E941F0301E00093522900E000936629C0
:103358000AE0009361290093602900E010E020E072
:1033680030E0EDE0F9E20083118322833383E1E06A
:10337800F9E200831183228333830093C22801E09A
:1033880010E0009386291093872901E000935F29B4
:1033980000E310E00E94960E02E00E941F0300E383
:1033A80010E00E94960E0CE00093502905E000936F
:1033B80051290BE000935C299CC081E090E00091CA
:1033C8004D2910E0F801EA5FFC4F049110E01A93D0
:1033D8000A9300913F291091402920914129309169
:1033E8004229021B130B1A930A939A938A93B0E00B
:1033F800BA93AA9323E332E207EC16E20E948239D9
:10340800289600EC0E94C60208E00E941F03E8E22A
:10341800F6E0008100FDF0CE0AE00E941F03409014
:10342800C9285090CA2800916D2910E01A930A9370
:103438007A926A925A924A9220E232E207EC16E2B3
:103448000E948239269600E80E94C60200918429CB
:1034580010918529013020E8120761F000E02091E1
:10346800842930918529213010E0310719F0006056
:10347800002311F0A0E001C0A1E0009145291091BE
:103488004629012B09F099CF80E090E098CF009170
:103498009029003119F402E000938E29B2D901E095
:1034A800C00E00E0D01E86016801093A21E6120725
:1034B80004F1CC24DD2400E00093400940D90091B8
:1034C800C9281091CA28083E23E0120718F401E021
:1034D8000093522900917029033058F0009158291F
:1034E800002339F442E0009170290E94C931009309
:1034F800582900917A29013001F500E000937A29D2
:1035080000EF11E00E94D605A02FAB3380F001EF49
:1035180011E00E94D605202F239501EF11E00E94AB
:10352800200620E000EF11E00E94200606C02A2FA6
:10353800239500EF11E00E94200600917B290230BC
:10354800A8F401EF11E00E94D605033078F001E0FD
:103558000093542900E0009379290FEF00935D2927
:1035680006E000935B2900E00093A40800915D2920
:10357800002309F085C30AE010916329011B009319
:103588007E2900917E2901301CF401E000937E29F8
:1035980000915F29013009F019C2E1EEF8E20081DB
:1035A800118122813381E9EFF8E2008311832283BC
:1035B8003383E5EEF8E20081118122813381E5E071
:1035C800F9E20083118322833383E5E0F9E2008185
:1035D8001181228133810E94E23228013901E9EF09
:1035E800F8E200811181228133810E94E232A80130
:1035F800B90100918E2910E0000F111F000F111F53
:10360800F801E35AF94D00811181228133810E942A
:10361800A233A801B901820193010E9485330E9457
:10362800EF32009347291093482940917E29542F5F
:10363800550F550B00914729109148290E94E731F1
:10364800212F220F220B322F0E94E2320E9438359E
:103658000E94EF320093492910934A2900917E294C
:10366800102F110F110B2091492930914A29021767
:1036780013070CF010C100915B29002309F00BC15E
:1036880000E0009360290091612903950093612966
:103698000F3118F001E000935229EDEFF8E20081B4
:1036A800118122813381E9EFF8E240815181628101
:1036B8007381401B510B620B730B408351836283F0
:1036C8007383E9E0F9E20081118122813381E5E029
:1036D800F9E24081518162817381401B510B620B79
:1036E800730B4083518362837383E9EFF8E20081AF
:1036F800118122813381E9EFF8E2408151816281B1
:1037080073810E942D3228013901E5E0F9E2008138
:10371800118122813381E5E0F9E2408151816281A2
:1037280073810E942D32A801B90182019301040F0F
:10373800151F261F371F0E94E2320E949D390E94E2
:10374800EF324801959487949594879499204AF488
:1037580027E000E81BEB0E945D0E00E21EE40E94D9
:10376800F40B009168290093692900914729109169
:103778004829212F220F220B322F0E94E2320E9469
:1037880038350E94EF32009357298401212F220FE8
:10379800220B322F0E94E2320E9438350E94EF320B
:1037A8000093C82800915829002321F408E00093C9
:1037B800562904C000915729009356290091582989
:1037C8000230E1F40091682910E0C80105E0402EBC
:1037D800552442E0009156290E94C93110E0401A50
:1037E800510AA2018C010E941932009369290091A3
:1037F8006929002319F401E000936929E5E0F9E259
:1038080000811181228133810E94E232A801B9012D
:103818002A013B01E9EFF8E200811181228133811D
:103828000E94E232A201B3010E94DE0E0093C12879
:103838000091C1280093C728009147291091482971
:10384800A016B10664F40091C1280093C3288092A1
:10385800862990928729A0904729B09048290091FD
:10386800C1281091C528011724F40091C12800939C
:10387800C4280091C4280093C5280091C328009348
:10388800C1280091772910916129011708F0F8C122
:103898000E940412F5C100917429002319F400E074
:1038A80000934009E9EFF8E2008111812281338118
:1038B800EDEFF8E20083118322833383E5E0F9E238
:1038C8000081118122813381E9E0F9E200831183CB
:1038D80022833383AA24A092C828BA2CBB0CBB0825
:1038E8000AE50093C4280091602903950093602994
:1038F80000E00093612900917429023009F0C0C1E9
:10390800E5E3F9E200811181228133810E94E232EC
:1039180028013901E1E3F9E2008111812281338133
:103928000E94E232A801B90100918E2910E0000F2F
:10393800111F000F111FF801E35AF94D0081118181
:10394800228133810E94A233A801B9018201930127
:103958000E9485330E94EF32212F220F220B322F33
:10396800E9E3F9E2008311832283338340907E29BF
:10397800542C550C5508652C752C42E050E060E03D
:1039880070E0E9E3F9E200811181228133810E942C
:103998008032401651066206730674F40091752948
:1039A800039500937529093008F46AC121E000E500
:1039B80016E40E945D0E64C100E00093752900E0E2
:1039C80010E000936A0910936B095AC1E1EEF8E21E
:1039D8000081118122813381E9EFF8E200831183AC
:1039E80022833383E5EEF8E200811181228133815D
:1039F800E5E0F9E20083118322833383E5E3F9E20A
:103A080000811181228133810E94E232280139012B
:103A1800E1E3F9E200811181228133810E94E232DF
:103A2800A801B90100918E2910E0000F111F000FA5
:103A3800111FF801E35AF94D008111812281338168
:103A48000E94A233A801B901820193010E94853323
:103A58000E94EF3200934729109348290091472983
:103A680010914829212F220F220B322F0E94E23277
:103A78000E9438350E94EF320093492910934A2951
:103A880000917E29102F110F110B20914929309197
:103A98004A29021713070CF0C8C000915B290023BC
:103AA80009F0C3C000E000936029009161290395E3
:103AB80000936129EDEFF8E20081118122813381C1
:103AC800E9EFF8E24081518162817381401B510B1B
:103AD800620B730B4083518362837383E9E0F9E2DD
:103AE8000081118122813381E5E0F9E24081518131
:103AF80062817381401B510B620B730B40835183AE
:103B080062837383E9EFF8E20081118122813381B6
:103B1800E9EFF8E240815181628173810E942D3280
:103B280028013901E5E0F9E2008111812281338120
:103B3800E5E0F9E240815181628173810E942D3272
:103B4800A801B90182019301040F151F261F371F11
:103B58000E94E2320E949D390E94EF3244E00E94A6
:103B6800FB31480199204AF427E004EF1EE70E9440
:103B78005D0E00E41CE90E94F40B009149290093B2
:103B880057290093562900915829002319F408E071
:103B98000093562900916129083068F1209156292F
:103BA800B22F80E49FE142E050E000914729109154
:103BB80048290E941932801B910B8C012B2F0E94DF
:103BC8005D0EE5E0F9E200811181228133810E94D6
:103BD800E232A801B9012A013B01E9EFF8E20081CC
:103BE8001181228133810E94E232A201B3010E9435
:103BF800DE0E0093C1280091472910914829A0168C
:103C0800B10664F40091C1280093C32880928629E4
:103C180090928729A0904729B09048290091C328FD
:103C28000093C5280093C1282BC000E000934009E9
:103C3800E9EFF8E20081118122813381EDEFF8E2AA
:103C48000083118322833383E5E0F9E20081118147
:103C580022813381E9E0F9E20083118322833383EF
:103C6800AA24BB2400E010E000938629109387293A
:103C780000E0009361290091602903950093602971
:103C880000916029003F41F010E000916129003F58
:103C980019F010601123A9F000E010E000938629C4
:103CA800109387290093C2280093C1288824809202
:103CB800C7288092C828982C990C990801E000938D
:103CC800522900915B29E8E3F3E00C94CD340C2DE4
:103CD8000F730023D9F40E94D90F802F4AE0082FD0
:103CE8000E94C93150E05A934A934AE0082F0E9433
:103CF800C93110E01A930A9327E832E207EC16E27A
:103D08000E94823924960DE80E94C6028091C1283B
:103D1800982F990F990B00918629109187290D5F8B
:103D28001F4F212F220F220B322F0E94E2320E94B6
:103D3800383540E050E060E87FEB0E9441330E9454
:103D4800EF32280100915729023020F0082F009304
:103D5800C22805C08091C228982F990F990B00910D
:103D68006129002309F08FC000915729023008F417
:103D78008AC0A2018C010E94193242E050E00E94E0
:103D88001932009380290091C328102F110F110BAD
:103D98002091C528322F330F330B021B130B0D5FF5
:103DA8001F4F212F220F220B322F0E94E2320E9436
:103DB80038350E94EF32380100918029102F110FF9
:103DC800110BA3010E94193200938029863500E067
:103DD80090073CF042E0009180290E94D73100937F
:103DE8008029E0917829F0E0F2968E179F077CF001
:103DF8000091782910E0015C1F4F081719073CF063
:103E080042E0009180290E94D731009380295520F3
:103E18001AF400E0009380290091802900231AF405
:103E280000E000938029009180290B301CF00AE003
:103E38000093802900918029102F110F110B2091D8
:103E48005C26322F330F330B021B130B42E050E07A
:103E58000E94193210915C26010F0093802900916D
:103E6800802900935C2600918029009381298C0188
:103E7800040D151D012B19F400E000938029009111
:103E8800802900937F2900916F29002309F0A2C09F
:103E9800C0FA6EF1109180290AE0109F002D0E944F
:103EA8004D11992362F05A924A929A938A932EE876
:103EB80032E207EC16E20E94823924960BC05A922D
:103EC8004A929A938A9327E932E207EC16E20E9413
:103ED8008239249603E80E94C60255200AF090C150
:103EE80007E80E94260203E20E946A0289C1009143
:103EF8005F29013009F043C0082F092B89F1992364
:103F080052F08C01045C1F4F4AE050E00E941932C5
:103F18000093C62803C005E00093C6280091C62870
:103F280000540E9426025520C2F09923B2F002E004
:103F3800401600E0500624F40FE50E946A0210C003
:103F480005E0401600E0500624F406E00E946A02EC
:103F580007C00FEF0E946A0203C003E20E946A02D0
:103F680000916029033308F44BC12FE932E207ECD2
:103F780016E20E94823903EC0E94C60241C1A42DB8
:103F8800A63008F0A5E02DEA32E207EC16E20E941E
:103F9800823903EC0E94C6020A2F0C530E942602A3
:103FA8000EE30E946A020FEC0A1B0E9426020CE331
:103FB8000E946A0255204AF42BEB32E207EC16E223
:103FC8000E94823904EC0E94C60200E21EE40E94AC
:103FD800F40B16C100916F290130F1F5C0FA26F0F3
:103FE800082F0E944D110CC1C201992032F403E23E
:103FF800402E552487E090E00BC000915F290023F4
:1040080021F40EE3402E552403C0552444244A9439
:10401800A0E008C00A2F08530E942602042D0E941F
:104028006A02A395B0E0A817B907A4F30091602924
:104038000F3148F028EC32E207EC16E20E94823990
:1040480007EC0E94C60207E80E9426020091802918
:10405800005D0E946A02D4C099238AF000918029E9
:10406800102F110F110B1A930A939A938A9322ED2A
:1040780032E207EC16E20E948239249615C00091BC
:104088008029102F110F110B1A930A934FEF5FEF2E
:104098008C010E94E7311A930A932EED32E207EC65
:1040A80016E20E948239249600E80E94C602C201E4
:1040B80099231AF483E290E006C0883000E0900764
:1040C80011F48FEF90E004E80E942602082F0E9466
:1040D8006A0200915F29013009F04BC00091602904
:1040E8000A3049F42AEE32E207EC16E20E948239DD
:1040F80000EC0E94C6020091C128013074F00091C2
:10410800C128102F110F110B045C1F4F4AE050E01B
:104118000E9419320093C62811C00091C128102F9F
:10412800110F110B42E050E00E9419320E5C1F4F34
:104138004AE050E00E9419320093C6280091C62830
:1041480000540E942602813000E090075CF0009144
:104158006029013020F006E00E946A0203C003E0F3
:104168000E946A0205EC0E9426020FE20E946A027F
:1041780047C043E084010E94FB31C801833C01E051
:10418800900734F400E099231AF00060002311F03E
:1041980082EC91E02BEF32E207EC16E20E948239C2
:1041A80000EC0E94C602A0E00FC00A2F07530E942D
:1041B80026020EE30E946A0206EC0A1B0E942602EF
:1041C8000CE30E946A02A3950A2F10E020E030E079
:1041D8000E94ED32280139018C01212F220F220B78
:1041E800322F0E94E2320E943835A801B9018201BB
:1041F80093010E94A434C8F200ED17E00E94F40B6A
:10420800C0FA1EF100913D2910E01A930A9300911B
:104218006B2910E01A930A930091632910E01A930E
:104228000A932CE033E207EC16E20E9482392696C4
:1042380008E80E94C602009163290A3031F409E8AF
:104248000E94260204E50E946A0218C580918F29FF
:1042580090E001969A938A9325E133E207EC16E2FF
:104268000E948239229600E80E94C60207E80E944E
:104278002602A0E009C00A2F10E000541E4F0E9439
:10428800D6050E946A02A395A930A8F300E21EE4AD
:104298000E94F40BE8E2F6E0008100FD6CC008E241
:1042A80010E00E94960E0DE00E942602A0E407E0AE
:1042B800009366290FC0009166290395009366292B
:1042C800003118F00FE000936629A0E408E210E03E
:1042D8000E94960E0091662900580E94260206E068
:1042E8000E941F03E8E0F6E0008102FFE4CFE8E067
:1042F800F6E0008101FD10C0009166290A9500933F
:104308006629073018F407E000936629A0E408E25C
:1043180010E00E94960EDECFE8E2F6E0008100FD94
:104328001EC0A3950A2FA02F0B3508F0A0E3AA33CF
:1043380009F4A0E20A2F0E946A0200916629005837
:104348000E94260202E310E00E94960E2A2F009196
:10435800662910E007541E4F0E942006BBCFE8E0F4
:10436800F6E0008103FDB6CF08E210E00E94960E49
:104378000CE00E9426020E94050C2EE133E207ECB5
:1043880016E20E94823900EC0E94C602A0E010C02A
:104398000A2F09530E9426020A2F0E946A02A83097
:1043A80031F40EEC0E9426020FEF0E946A02A395D8
:1043B80080918F2990E00196B0E08A179B0744F717
:1043C8005DC40E94D90FC8014AE050E08C010E94E8
:1043D80019325A934A934AE050E08C010E941932EC
:1043E8001A930A932FE233E207EC16E20E9482390D
:1043F800249600E80E94C6024AE0009162290E94C1
:10440800C93150E05A934A934AE0009162290E94C8
:10441800C93110E01A930A9322E433E207EC16E25A
:104428000E948239249600EC0E94C60200914F290E
:10443800002321F408E80E94260203C008EC0E9429
:1044480026020EE30E946A0202E00E941F0316C4BD
:1044580000916A2910E01A930A9325E533E207ECE4
:1044680016E20E948239229600E80E94C60227E6D8
:1044780033E207EC16E20E94823900EC0E94C60281
:10448800A0E010C00A2F0A530E9426020A2F0E9499
:104498006A02A83031F40EEC0E9426020FEF0E9447
:1044A8006A02A39500916A290A1760F702E00E9440
:1044B8001F03E4C30E946B0FC8019A938A9329E7EC
:1044C80033E207EC16E20E948239229600E80E9445
:1044D800C6020091CD281091CE281A930A932CE891
:1044E80033E207EC16E20E948239229609E80E941C
:1044F800C6024091BF285091C0284F5F5F4F652F7B
:10450800660F660B762F00E01CE62CED32E00E9469
:10451800803248E050E060E070E00E9480323A93D8
:104528002A931A930A9325E933E207EC16E20E94CC
:104538008239249600EC0E94C60200E21EE40E9422
:10454800F40B9CC340E250E060E070E0E5EEF8E276
:1045580000811181228133810E9480320E940D0FD7
:1045680025EA33E207EC16E20E94823900EC0E9449
:10457800C6020FED10E01A930A9300913F2910919B
:1045880040291A930A9320EB33E207EC16E20E94C3
:10459800823924960AEC0E94C60200E21EE40E94B8
:1045A800F40B01E00093542900E0009379290CE012
:1045B800009350290E941C3861C300917B29023066
:1045C80031F400E00093542907E000935B2900913F
:1045D8005429002309F44DC00E949F140BEE11E0EA
:1045E8000E94D605902F80E00CEE11E00E94D605BF
:1045F80010E0802B912B8093D5289093D62800EF3C
:1046080011E00E94D605802F01EF11E00E94D60527
:104618002091D5283091D6283A932A9390E09A93FE
:104628008A9310E01A930A9329EB33E207EC16E217
:104638000E948239269600E80E94C6020091D72877
:104648001091D8281A930A932FEC33E207EC16E25C
:104658000E948239229600EC0E94C60200915029DD
:1046680000540E94260200E0009354290DE00E94A5
:10467800260202E00E941F0301C300915A29002369
:1046880011F4A3E501C0ADE40E946B0F1A930A93DD
:1046980022EE33E207EC16E20E948239229600E805
:1046A8000E94C602B0E0BA93AA932BEE33E207EC5D
:1046B80016E20E948239229606E80E94C60227EF77
:1046C80033E207EC16E20E94823900EC0E94C6022F
:1046D800A0E010C00A2F0A530E9426020A2F0E9447
:1046E8006A02A83031F40EEC0E9426020FEF0E94F5
:1046F8006A02A39500916E290A1760F700E21EE48A
:104708000E94F40BBBC200914D2910E0F801EA5F4A
:10471800FC4F049110E01A930A9328E034E207EC66
:1047280016E20E948239229600E80E94C60224E11D
:1047380034E207EC16E20E94823909E80E94C602B8
:104748002CE134E207EC16E20E94823900EC0E9468
:10475800C602A0E010C00A2F07530E9426020A2FA3
:104768000E946A02A83031F40EEC0E9426020FEF74
:104778000E946A02A39500914D290A1760F700E28A
:104788001EE40E94F40B7AC201E00E94CF1300914C
:10479800C9281091CA2801382CE0120730F002E02D
:1047A8001DE00093C9281093CA280091C9281091C8
:1047B800CA281A930A932DE234E207EC16E20E9403
:1047C8008239229600E80E94C6020091452910917C
:1047D80046291A930A9328E334E207EC16E20E946A
:1047E8008239229609E80E94C6020FED10E01A935A
:1047F8000A9300914329109144291A930A9321E4BA
:1048080034E207EC16E20E948239249600EC0E94FA
:10481800C60200914F29002321F409E80E942602CC
:1048280003C009EC0E9426020EE30E946A0200E21D
:104838001EE40E94F40B22C200E00093832924E5C1
:1048480034E207EC16E20E94823900E80E94C602B0
:1048580000917C29007F002351F422E634E207EC22
:1048680016E20E9482390DE80E94C60206C026E6BA
:1048780034E207EC16E20E9482390DE80E94C60273
:104888002AE634E207EC16E20E94823900EC0E9424
:10489800C60200917C290F70002351F422E634E20D
:1048A80007EC16E20E9482390DEC0E94C60206C08F
:1048B80026E634E207EC16E20E9482390DEC0E94EB
:1048C800C60204E00E941F03D9C100E00093060954
:1048D80000915829002311F4ADE20BC0009158292A
:1048E800013011F4AFE205C000915829023009F4F3
:1048F800ACE7B0E0BA93AA9328E734E207EC16E2F3
:104908000E948239229600EC0E94C602A0E010C0E4
:104918000A2F09530E9426020A2F0E946A02A83011
:1049280031F40FEC0E9426020FEF0E946A02A39551
:10493800009167290A1760F780E090E0A0E005C0C1
:104948000E94F80F800F911FA395AA30C8F34AE080
:1049580050E08C010E941932C80100919300033085
:1049680008F4839700EF11E00E94D605402E01EF6E
:1049780011E00E94D605202F0FED10E01A930A933C
:104988009A938A9355245A924A9230E03A932A93FA
:104998002BE834E207EC16E20E948239289600E8F8
:1049A8000E94C60202E00E941F0301E000935429FE
:1049B80065C100916C29053009F052C00091542955
:1049C800002309F499C00091512910E0F801E25F31
:1049D800F74DA081AA2341F04A2F50E000E41CE9DA
:1049E8000E940132C80102C080E090E027EA34E268
:1049F80007EC16E20E94823900E80E94C6029A93E8
:104A08008A9328EB34E207EC16E20E948239229658
:104A180000EC0E94C60222E04A2F50E006E910E0AE
:104A28000E94E7310E945D0E0091512900540E94B6
:104A3800260200918329002321F400E20E946A02E1
:104A480003C00FEF0E946A020091512900540E948E
:104A580026020EE00E94260200E0009354294CC072
:104A680000916C29033030F480916C2990E0880F14
:104A7800991F09C000916C29033019F48AE090E06D
:104A880002C08AE590E09A938A9329EC34E207EC15
:104A980016E20E948239229600E80E94C60200911E
:104AA800742910E0000F111FF801EA5DFC4F059111
:104AB80014911A930A9322ED34E207EC16E20E944D
:104AC8008239229607E80E94C6022BED34E207ECF1
:104AD80016E20E94823900EC0E94C602A0E008C0DB
:104AE8000A2F0E946A020A2F06530E942602A395E3
:104AF80000916C290A17A0F702E00E941F03BEC0AC
:104B080000E0009383290091702910E0000F111F25
:104B1800F801EF5EFC4F059114911A930A932CEE5D
:104B280034E207EC16E20E948239229600E80E94DD
:104B3800C6022DEF34E207EC16E20E94823900EC3F
:104B48000E94C602A0E008C00A2F06530E9426024F
:104B58000A2F0E946A02A395009170290A17A0F7EC
:104B680002E00E941F038AC000916F2910E0000F25
:104B7800111FF801E55EFC4F059114911A930A93F1
:104B88002EE035E207EC16E20E948239229600E810
:104B98000E94C60226E135E207EC16E20E9482393D
:104BA80000EC0E94C602A0E008C00A2F06530E942B
:104BB80026020A2F0E946A02A39580916F2990E02D
:104BC8000196B0E08A179B0784F702E00E941F0352
:104BD80001E00093542952C0009154290023A1F107
:104BE80027E235E207EC16E20E94823900E80E94CB
:104BF800C602A0E004C000E20E946A02A395A031A8
:104C080090F40A2F00540E9426024A2F009184290A
:104C1800109185290E94FB310170002361F303E2A2
:104C28000E946A02EBCF05EC0E9426020FE20E9466
:104C38006A020091662900540E9426020EE00E9432
:104C4800260200E00093542908EE1DEF0E94F40BA1
:104C580015C000E00093832928E335E207EC16E24B
:104C68000E94823900E80E94C60229E435E207EC76
:104C780016E20E94823900EC0E94C60200E000930E
:104C88003E29E8E0F6E0008103FDC0C00E94FB1465
:104C980000914D290E94CF1301E00093522903E0AF
:104CA800009306090CE00E94260200915929013060
:104CB80099F40EE110E00E94960EE8E0F6E000811B
:104CC80003FFFBCF04EB009361290093602900E008
:104CD800009359290C940731E8E0F6E0008103FDC0
:104CE8004BC008EE1DEF0E94F40B00913E2903957E
:104CF80000933E298091D3289091D428039610E000
:104D08008017910748F700915D29009500935D2968
:104D180001E00093592900E00093832900915D295F
:104D28000023C9F400E000935B292AE535E207EC8B
:104D380016E20E94823900EC0E94C60202E00E943C
:104D48001F0300916F29023011F00E94290C0EE315
:104D5800C02EDD2406C000915C2900935B290E94C7
:104D6800050C01E00093542900E000935E290AE550
:104D780010E00E94960E82C100915D290023A1F4E3
:104D880000915F29013021F400E000935F2903C0FE
:104D980001E000935F2901E00093522904EB00939E
:104DA8006129009360292CC000915E29013059F4D3
:104DB80000915B29039500935B290930E8F001E035
:104DC80000935B2919C000915E29023059F40091C3
:104DD8005B29039500935B290B3070F007E0009383
:104DE8005B290AC000915B29039500935B29013177
:104DF80018F00BE000935B2900915B2900935C2974
:104E080008E210E00E94960E0C940431E8E2F6E005
:104E1800008100FDCDC400E00093400900915B29AA
:104E28000050E1F0025009F488C1025009F493C11E
:104E38000A9509F4E1C10A9509F4F8C20A9509F43A
:104E480075C3025009F4CAC3025009F4F5C30A95A0
:104E580009F434C4035009F464C4A2C401E00E94F4
:104E6800260201E00E94CF1300E41CE90E94F40B23
:104E7800E8E2F6E0008100FD11C000E61AEE0E94AB
:104E8800F40B00913E29039500933E292091D328E5
:104E98003091D42810E02017310750F700913E29AF
:104EA800039500933E292091D3283091D42810E00F
:104EB8002017310708F0E8C0EDEEF8E20081118113
:104EC800228133810E94E232A801B901CA01DB01C3
:104ED800E9EEF8E200811181228133810E94E232F9
:104EE800AC01BD010E94D30E0093C128E9EEF8E29F
:104EF8000081118122813381E9EEF8E240815181FC
:104F0800628173810E942D32C801D901EDEEF8E269
:104F18000081118122813381EDEEF8E240815181D7
:104F2800628173810E942D32A801B9018C019D0113
:104F3800040F151F261F371F0E94E2320E949D3959
:104F48000E94EF3248018401000F111F212F220F08
:104F5800220B322F0E94E2320E9438350E94EF3233
:104F6800A02FAF3F09F4AAE0A83020F40091C1288F
:104F7800073B24F003E000936B290DC0A43020F414
:104F88000091C1280D3A24F002E000936B2903C078
:104F980001E000936B290091C128053C44F410E01E
:104FA8000091C128063A1CF01060112391F02BE6FD
:104FB80035E207EC16E20E94823900EC0E94C60234
:104FC80000EA10E00E94960E00EB10E00E94960E98
:104FD80037C0EDEEF8E200811181228133810E9411
:104FE800E23228013901E9EEF8E2008111812281DB
:104FF80033810E94E232A801B901820193010E9423
:105008001B3440918E2950E0440F551F440F551F03
:10501800FA01E35AF94D00831183228333832CE785
:1050280035E207EC16E20E94823900EC0E94C602C3
:1050380000E510E00E94960E00E210E00E94960E35
:1050480000916B2910E01A930A930091C128102F40
:10505800110F110B1A930A93B0E0BA93AA9329EB94
:1050680035E207EC16E20E948239269600E80E9493
:10507800C602E8E2F6E0008100FFFBCF00914D296F
:105088000E94CF130C94043101E00093522900913F
:10509800C9281091CA2801382CE0120730F004EE14
:1050A8001CE00093C9281093CA280091C9281091C0
:1050B800CA281A930A932DE835E207EC16E20E94F3
:1050C8008239229600E80E94C60200EF11E00E9491
:1050D800D605802F01EF11E00E94D60590E09A9343
:1050E8008A9310E01A930A932FE935E207EC16E247
:1050F8000E948239249600EC0E94C60200E310E068
:105108000E94960E00916129002311F401E001C06C
:1051180000E00093602900914D290E94CF1304E11B
:105128000E941F0322EB35E207EC16E20E94823947
:1051380000EC0E94C6020C94043100914F2900959E
:1051480000934F290AE00E941F0300E510E00E9427
:10515800960E0C94043166247724442455240E9426
:10516800C60E8BE291E013C080932609909327091D
:1051780003E00E941F030E946B0F38014614570476
:105188002CF423018093BF289093C0280A968D3E63
:1051980002E090074CF30091BF281091C0280093BB
:1051A8002609109327090E94181310E400E50E94AD
:1051B800BA0E3091C028232F01E010E00E9420068B
:1051C8002091BF2802E010E00E9420060C940431D0
:1051D8002FEE35E207EC16E20E94823900E80E94C1
:1051E800C60200E810E00E94960E00E810E00E9457
:1051F800960E0AE00E941F03E8E2F6E0008100FD37
:10520800FFC000E61AEE0E94F40B00913E290395B8
:1052180000933E292091D3283091D42810E02017FC
:10522800310750F701E00093552900E010E00093A2
:105238003F29109340290E94401001E00093522911
:105248002DEC35E207EC16E20E94823900E80E9454
:10525800C60200E310E00E94960E01E00093522976
:105268000091D328102F02E0109F002D0E941F03E9
:105278002EED35E207EC16E20E94823900E80E9422
:10528800C60200E310E00E94960E0091D328102F6A
:1052980002E0109F002D0E941F0380E090E0A0E034
:1052A8001EC0EDEEF8E200811181228133810E9457
:1052B800E232A801B9012A013B01E9EEF8E20081D6
:1052C8001181228133810E94E232A201B3010E943E
:1052D800D30E800F911F07E00E941F03A395AA30E9
:1052E80000F34AE050E08C010E941932C80106EA36
:1052F8001FEF081B190B00933F29109340290091B9
:105308003F2910914029093621E0120744F0EFE3C4
:10531800F9E2008111810856114000831183109130
:105328004029112342F4EFE3F9E200811181085981
:105338001E4F008311830E94401001E00093522900
:105348000091D3280E941F03EDEEF8E2008111813D
:10535800228133810E94E232A801B9012A013B016E
:10536800E9EEF8E200811181228133810E94E23264
:10537800A201B3010E94D30EC8018C01AC010E94A6
:10538800E731212F220F220B322F0E94E2320E9496
:105398009D3940E050E060EB72E40E94A43408F4C8
:1053A80017CF20E036E207EC16E20E94823900E8C7
:1053B8000E94C60205E210E00E94960E05E00E94D7
:1053C8001F0305E210E00E94960E30914029232F1A
:1053D80005E010E00E94200620913F2906E010E039
:1053E8000E94200630914229232F07E010E00E94F6
:1053F80020062091412908E010E00E942006FCCEFA
:1054080000915529002389F421E136E207EC16E2E0
:105418000E94823900E80E94C60208EE1DEF0E9431
:10542800F40B00E510E00E94960EEAC6E8E2F6E00A
:10543800008100FD11C008EE1DEF0E94F40B0091E1
:105448003E29039500933E292091D3283091D428F2
:1054580010E02017310750F700913E29039500937B
:105468003E292091D3283091D42810E02017310705
:1054780008F064C00091D5281091D6280E94DD1448
:105488002091D7283091D8280217130721F523E255
:1054980036E207EC16E20E94823905EC0E94C60249
:1054A80000E210E00E94960E00E510E00E94960EC1
:1054B8003091D828232F0DEE11E00E94200620916C
:1054C800D7280EEE11E00E94200627E303EF11E033
:1054D8000E9420061EC029E236E207EC16E20E946E
:1054E800823900E80E94C6022AE336E207EC16E297
:1054F8000E94823900EC0E94C60200E011E00E947E
:10550800960E00E211E00E94960E00E411E00E945F
:10551800960EE8E2F6E0008100FFFBCF08EC0E945F
:105528001F0308ED04BF01E00093790000915A2998
:105538000023D1F501E000935A2939C00091502980
:1055480010E0F801ED5FF74D008103950F70209191
:10555800502930E0F901ED5FF74D008320910F28C5
:10556800322F20E0330F330F330F330F10911028F1
:1055780000E0202B312B0091112810E044E00E941C
:10558800EF31202B312B0091122810E0202B312BEA
:105598002093D7283093D8280CE310E00E94960E69
:1055A80001E0009354292CC600E000935A29409149
:1055B8006E2950E00FEF10E00E94E7310E94AB0C1B
:1055C80020915A2904EF11E00E94200602E310E01E
:1055D8000E94960E04E00E941F0312C6E8E2F6E05D
:1055E800008100FD1CC008EE1DEF0E94F40B009125
:1055F8003E29039500933E292091D3283091D42841
:1056080010E02017310750F700E610E00E94960ED0
:105618000E94580D10E200E30E94BA0E2FCD0091AF
:105628004F29009500934F2902E310E00E94960E3F
:1056380005E00E941F03E4C5E8E0F6E0008102FDF2
:1056480010C0009182290395009382292091822914
:105658000AEE11E00E9420060EE110E00E94960E6C
:1056680025C0E8E0F6E0008101FD10C00091822924
:105678000A9500938229209182290AEE11E00E945E
:1056880020060EE110E00E94960E10C000915829E5
:10569800039500935829033018F000E00093582927
:1056A8002091582908EF11E00E9420060CE00E9482
:1056B8001F0302E310E00E94960EA2C500916C2918
:1056C8000530B9F400918329009500938329A091AE
:1056D8005129A550B0E0FD01ED5EF74D20810A2F5C
:1056E80010E000571E4F0E94200601E00093542945
:1056F80010C000917429039500937429033018F0A1
:1057080000E0009374292091742902EF11E00E94AF
:10571800200602E310E00E94960E06E00E941F0396
:105728006FC581E090E0409166298C010E94EF31BD
:10573800C8014091662900918429109185290E9409
:10574800FB310170002379F080959095E4E8F9E247
:1057580000811181082319230083118310E500E4D7
:105768000E94BA0E0CC0E4E8F9E200811181082B0E
:10577800192B0083118310E300E40E94BA0E01E0A4
:1057880000935429209184290AE010E00E94200601
:1057980030918529232F0BE010E00E94200630C5A8
:1057A80001E00093522908E210E00E94960E28C5F5
:1057B800E8E0F6E0008102FDAEC200E00093400997
:1057C80000915B29E0E6F3E00C94CD34E8E0F6E0E4
:1057D800008102FD29C000E61AEE0E94F40B009138
:1057E8003E29039500933E292091D3283091D4284F
:1057F80010E02017310750F70091642900950093B5
:1058080064292091642909EF11E00E94200601E033
:105818000093552900E510E00E94960E01E00E94D1
:105828001F030E941B15EFC400915529002389F519
:10583800009163290395009363290B3018F00AE05F
:105848000093632900917029033038F0009163298F
:105858000A3019F409E0009363292091632903E0D1
:1058680010E00E942006009163290A3049F400EDF7
:1058780017E00E94AB0C10E500E70E94BA0E3FC289
:1058880040916E2950E00FEF10E00E94E7310E942E
:10589800AB0C35C200918F29039500938F290430F2
:1058A80018F003E000938F290E94E31320918F29B9
:1058B8000AEF11E00E94200622C200914F2900231E
:1058C80089F000916229039500936229043618F043
:1058D80003E600936229209162290EEF11E00E94ED
:1058E800200610C0009165290A95009365290A30A1
:1058F80018F40AE000936529209165290CEF11E05E
:105908000E94200600E315E70E94F40BF8C10091FD
:105918006A29039500936A29093018F008E0009372
:105928006A290BE910E000932608109327082091B4
:105938006A290DEF11E00E94200680916A2990E003
:10594800019680932A0890932B08D9C18091BF288B
:105958009091C02801978093BF289093C0288B32DC
:1059680001E0900734F40BE211E00093BF28109394
:10597800C0280091BF281091C028009326091093D1
:1059880027090E9418133091C028232F01E010E046
:105998000E9420062091BF2802E010E00E94200605
:1059A800AEC180913F2990914029019680933F296B
:1059B80090934029883601E0900734F000E010E029
:1059C80000933F29109340290E94401030914029AC
:1059D800232F05E010E00E94200620913F2906E0D1
:1059E80010E00E94200630914229232F07E010E0A2
:1059F8000E9420062091412908E010E00E9420061C
:105A08007EC100915029039500935029003118F068
:105A18000FE00093502900E00093792901E00093FA
:105A2800542902E00E941F036AC100916E29039560
:105A380000936E29093018F008E000936E29409110
:105A48006E2950E00FEF10E00E94E7310E94AB0C86
:105A580020916E290CE010E00E94200650C10091B0
:105A68004D29039500934D29053018F004E0009363
:105A78004D2900914D290E94CF1320914D2904E111
:105A880010E00E9420063BC1E8E0F6E0008101FD3D
:105A98001BC000E010E000934529109346290093AD
:105AA80043291093442904E610E00E94960E06E06C
:105AB8000E941F0320E00EE010E00E94200620E074
:105AC8000FE010E00E94200600914F29002309F5FD
:105AD8008091452990914629019680934529909374
:105AE8004629813008E0900734F000E018E0009380
:105AF80045291093462930914629232F00E110E0CB
:105B08000E9420062091452901E110E00E9420060C
:105B180020C080914329909144290196809343297C
:105B280090934429883601E0900734F000E010E0B3
:105B3800009343291093442930914429232F0EE0E0
:105B480010E00E942006209143290FE010E00E94F7
:105B5800200620914529309146290091432910912A
:105B680044290E94030D02E00E941F03C8C000914F
:105B78007C290F70002331F400917C290F60009379
:105B88007C2905C000917C29007F00937C290E9414
:105B98001B1520917C2909EE11E00E9420060CE0DB
:105BA8000E941F03ACC000916729039500936729E1
:105BB800093018F008E000936729009167290093DD
:105BC80068292091672906EF11E00E94200697C0F6
:105BD80000916C290530B9F000916C290395009368
:105BE8006C29053030F005E000936C2905E000933E
:105BF800512920916C2907EF11E00E94200601E04D
:105C0800009354292CC000918329002359F4009152
:105C180051290395009351290F30E8F00EE00093C5
:105C2800512919C00091512910E0F801E25FF74DA0
:105C380000810A952091512930E0F901E25FF74D82
:105C48000083083040F408E02091512930E0F90140
:105C5800E25FF74D008300E61AEE0E94F40B01E0C4
:105C6800009354294CC00091702903950093702922
:105C7800053018F004E0009370292091702903E1A1
:105C880010E00E9420060E94181302E00E941F03E1
:105C980036C000916F29039500936F29033018F0DF
:105CA80002E000936F2920916F2905EF11E00E940F
:105CB800200600E61AEE0E94F40B21C00091662926
:105CC800039500936629003118F000E000936629D7
:105CD80001E00093542913C02BE436E207EC16E2E6
:105CE8000E94823900E80E94C60200E510E00E9486
:105CF800960E0FE00E941F0307E000935B290091B6
:105D08008329002321F408E210E00E94960E01E0A6
:105D18000093522975C2E8E0F6E0008101FD70C2E7
:105D280000E00093400900915B29E8E8F3E00C9457
:105D3800CD34E8E0F6E0008101FD2CC000E513EC6D
:105D48000E94F40B00913E29039500933E2920916F
:105D5800D3283091D42810E02017310750F700914C
:105D68006B29039500936B29043018F001E0009328
:105D78006B2920916B290DE010E00E94200601E0BC
:105D88000093552900E510E00E94960E02E00E945B
:105D98001F0339C200915529002311F50091632989
:105DA8000A95009363290F3F19F400E000936329D3
:105DB8002091632903E010E00E94200600916329E6
:105DC800002329F400E010E00E94AB0C0EC24091C1
:105DD8006E2950E00FEF10E00E94E7310E94AB0CF3
:105DE80004C200918F290A9500938F290F3F19F457
:105DF80000E000938F290E94E31320918F290AEF76
:105E080011E00E942006F1C100914F29002389F07A
:105E1800009162290A95009362290F3F19F400E066
:105E280000936229209162290EEF11E00E9420065A
:105E380010C000916529039500936529013518F074
:105E480000E500936529209165290CEF11E00E9477
:105E5800200600E315E70E94F40BC7C100916A29E8
:105E68000A9500936A290F3F19F400E000936A2904
:105E780020916A290DEF11E00E94200680916A297D
:105E880090E0019680932A0890932B08AEC18091E8
:105E9800BF289091C02801968093BF289093C0286E
:105EA8008E3E02E0900734F00DEE12E00093BF281A
:105EB8001093C0280091BF281091C028009326098C
:105EC800109327090E9418133091C028232F01E04E
:105ED80010E00E9420062091BF2802E010E00E94F6
:105EE800200683C180913F29909140290197809392
:105EF8003F2990934029992332F408E611E0009352
:105F08003F29109340290E94401030914029232FA7
:105F180005E010E00E94200620913F2906E010E0ED
:105F28000E94200630914229232F07E010E00E94AA
:105F380020062091412908E010E00E94200655C162
:105F4800009150290A95009350290C3018F40CE060
:105F58000093502900E00093792901E00093542927
:105F680002E00E941F0341C100916E290A95009327
:105F78006E290F3F19F400E000936E2940916E29B5
:105F880050E00FEF10E00E94E7310E94AB0C209127
:105F98006E290CE010E00E94200627C100914D29CF
:105FA8000A9500934D29013018F401E000934D291A
:105FB80000914D290E94CF1320914D2904E110E052
:105FC8000E94200612C1E8E0F6E0008102FD11C03F
:105FD80000E010E0009345291093462900934329D7
:105FE8001093442904E610E00E94960E06E00E94F1
:105FF8001F0300914F290023F9F4809145299091BE
:10600800462901978093452990934629992332F48C
:1060180000E010E000934529109346293091462965
:10602800232F00E110E00E9420062091452901E17C
:1060380010E00E9420061EC08091432990914429B7
:1060480001978093432990934429992332F407E6D2
:1060580011E0009343291093442930914429232FB8
:106068000EE010E00E942006209143290FE010E086
:106078000E94200620914529309146290091432904
:10608800109144290E94030D02E00E941F03ADC035
:1060980000917C29007F002331F400917C29006F56
:1060A80000937C2905C000917C290F7000937C29FE
:1060B8000E941B1520917C2909EE11E00E94200600
:1060C8000CE00E941F0391C0009167290A95009374
:1060D80067290F3F19F400E00093672900916729A9
:1060E800009368292091672906EF11E00E94200695
:1060F8007CC000916C290530A1F000916C290A95AB
:1061080000936C29013018F401E000936C29209168
:106118006C2907EF11E00E94200601E00093542942
:1061280064C000918329002371F4009151290A95D4
:10613800009351290530C8F404E000936C290CE061
:106148000E94260212C00091512910E0F801E25F76
:10615800F74D0081002349F00091512910E0F80122
:10616800E25FF74D00810395008300E61AEE0E9476
:10617800F40B01E00093542938C0009170290A9566
:1061880000937029002319F401E0009370292091ED
:10619800702903E110E00E9420060E94181302E013
:1061A8000E941F0322C000916F290A9500936F294E
:1061B8000F3F19F400E000936F2920916F2905EF34
:1061C80011E00E94200600E61AEE0E94F40B0DC0B2
:1061D800009166290A95009366290F3F19F40FE08C
:1061E8000093662901E00093542900918329002334
:1061F80021F408E210E00E94960E01E00093522973
:1062080000E0009355298091480690E080739070D3
:106218000091902910E00817190711F40C94531AEB
:106228008093902900919029003329F400E000938D
:106238008E290C94521A00919029003211F00C9476
:106248004B1A01E000938E290C94521A000088958D
:10625800FECF0E941A35C801D9012A013B015CD042
:1062680057D071F48201930153D051F401E2E8E967
:10627800F9E2008341830FEF1FEF2FE73FE73DC0AF
:1062880044D0A201B3010E944133AC01BD0140D00A
:1062980061F442D03AD00E94BC340BED1FE029ECE7
:1062A80010F43FE32AC03FEB28C0A201B3012DD070
:1062B8000E941B34080119012FD0820193010E940A
:1062C800A43423D0A0F41CD050F424D0A801B901E0
:1062D8000BED1FE029E430E40E9485330EC01AD08C
:1062E8004BED5FE069E470EC0E94413306C008D0D2
:1062F80010F410D002C00ED03058E8E00C942B35C2
:106308000E94BC348001910108958C019D0108957B
:106318000C949A340C94333840E050E060E070E01C
:1063280008953F7741E00C94D23803E20DBF01E2B3
:106338000EBFC0E0D1E20E94BB35002311F00E94DD
:10634800B5380E945E150E942A310C942A310D013D
:10635800DA0140E050E060E070E00E949A3439F4DD
:1063680000E010E04D934C9320E030E00CC0B90100
:10637800660F771F7E57572F550F550B7D935C93EC
:106388002F7730783F63D00108950024E8E0EA953C
:1063980032F0001F001C0416D0F3041AF8CF001FB7
:1063A800402D00950895FF27442312F4F16041958C
:1063B800002312F4F09501950E94C931F0FD019572
:1063C800F1FD41950895149F102D059F100D049F10
:1063D800002D110D08954A951AF0000F111FFBCFDB
:1063E80008954A951AF016950795FBCF08954A9592
:1063F8001AF015950795FBCF089500241124EFE0B6
:10640800001F111F001C111C0416150610F0041A99
:10641800150AEA95AAF7001F111FA001009510950B
:1064280008955195419550400895FF27552312F43A
:10643800F160F7DF112312F4F09507D00E940132C2
:10644800F0FD03D0F1FDEDCF0895119501951040B1
:1064580008952224349F302D259F300D169F300D2E
:10646800079F300D249F202D310D159F200D311DC4
:10647800069F200D311D149F102D210D321D059FE3
:10648800100D211D321D049F002D110D221D321DDE
:1064980008954A952AF03695279517950795F9CFC7
:1064A80008954A952AF03595279517950795F9CFB8
:1064B8000895002411241001E0E2EA9592F0001FEB
:1064C800111F221F331F001C111C221C331C041611
:1064D80015062606370688F3041A150A260A370A07
:1064E800ECCF001F111F221F331FA001B10100951F
:1064F8001095209530950895FF27772312F4F160C1
:1065080015D0332312F4F09509D00E945D32F69528
:1065180008F404D0F69508F409C00895309520953C
:10652800109501951F4F2F4F3F4F08957095609517
:10653800509541955F4F6F4F7F4F0895FF27112466
:1065480077FB660F771F089409F4771F679517F88C
:10655800EE27002437FB220F331F089409F4331F5A
:10656800279507F8089527FD0EC0EE0F001F111F8D
:10657800221F3A953230B8F7332319F427FD31E05A
:1065880002C027FF30E0E03821F400FF08940EF441
:1065980088940F4F1F4F2F4F3F4F323038F433231B
:1065A80019F427FD31E002C027FF30E03F3F29F012
:1065B800220F000C379527950895ACC0032E0020B4
:1065C80012F40E949232E02F012F122F232F3EE95E
:1065D800D1CF0024F8CFBCDF432F4F5748F04F31BD
:1065E80048F007FC91C03FE72FEF1FEF0FEF08952A
:1065F80033278CC0322F212F102F0E2F4F5141954A
:106608000E944D3207FE08950C949232F901EE0F64
:10661800FF1F37FBFF3F31F0EF2BE12BE02B889476
:10662800B8940895E02BE12B21F008949894B8943D
:1066380008959894889438940895FB01EE0FFF1FED
:1066480077FBFF3F31F0EF2BE52BE42B8894B894D0
:106658000895E42BE52B69F3E8CFEFDF68F021F428
:106668003723262F8A010895372FFBCFE6DF20F046
:106678000BF008957327EAF751C0C8DFE8F3B3F3C6
:1066880061F3DBDFC8F383F3A1F358DF4017510749
:106698006207730731F4011411F10024E894889417
:1066A8002BC078F0332E372F732D322E262F632DE3
:1066B800312E152F532D302E042F432D302C012C25
:1066C800132C371739F0669557954795F795E0409D
:1066D8007395F7CFE7FBEE0FE0E010246AF0EF0FB9
:1066E800041F151F261F60F4279517950795E79532
:1066F80008F4689433953ECFEF0B040B150B260B6B
:1067080039CFE0E87E27B9CF302D307822271127FE
:10671800002708953FE7302920E8F9CF3FEF2FEF12
:10672800F6CF8BDFD8F3D1F370783727089585DF5C
:10673800A8F3A3F3F9CF3078372793CF67DF70F347
:1067480083F3A9F37ADF50F3B3F3A9F3F7DE012457
:10675800E8943F57E040370FEF1F12F0D9F603C017
:106768003A3E90F26894E0E00A92AA933A93AA27F4
:10677800332422243327049FF001059FF00D712D47
:10678800731F149FF00D711D221C069F700D211C94
:10679800331C159F700D211C331E249F700D211C66
:1067A800331E169F200C311CAA1F259F200C311C5C
:1067B800A31F269F300CA11D39915EF43395A69531
:1067C800379427947795F795E79533953130BCF34F
:1067D80016C0AA2322F0332351F4339510C0339501
:1067E80071F4A991099096CFA7FD09C03A95EE0FCB
:1067F800FF1F771F221C331CAA1F3230A8F7E8940A
:10680800FE2B09F068942A2F8101E72FA99109909E
:10681800BACE13DF10F00BF087CF80CF0EDFE9F38D
:10682800E0F3032E072670CF032E072673CFEEDE84
:10683800A0F37BF399F301DF80F39BF3A9F37EDEEA
:10684800012427FD06C0000F111F221F3150E04010
:10685800F8CF67FD06C0440F551F661F7150F04002
:10686800F8CFE894371BEF0B3158EF4F2AF0EE239F
:10687800E9F63F3FD9F203C03A3EA8F26894E0E057
:10688800F0E01124139440175107620738F0315093
:1068980008F46894000F111F221FEE1F041B150B2C
:1068A800260BEF0B000F111F221FEE1F0A9279E132
:1068B8007A95AAF0041715072607EF0730F0041B8E
:1068C800150B260BEF0B089401C08894111C221C91
:1068D800331C001C000F111F221FEE1FE9CFF0F917
:1068E800E894E22BE12BE02B09F0689406943794A6
:1068F80027941794E79508F468947395B9F3099069
:10690800332311F0F0FF09C0369427941794E795C4
:1069180008F4689433953130BCF3012D122D232DE2
:1069280032CE8BCE98940895189408956FDED0F3E4
:10693800C1F383DEB8F30417150726073707089550
:106948007CDEA0F063DE90F029F0E32FE7273AF42D
:106958007317089572DE51F04EF0089408950417E5
:1069680015072607370719F016F4B8F7889408951D
:1069780064DEE0F34BDED0F3E7DFC0F3089408955C
:106988007591659155914591159011FA259035901D
:106998000895F9DF041B10E003C0F4DF041B150B96
:1069A80020E030E005C0ECDF041B150B260B370B8D
:1069B800B8F010FC17C045910590E00FF11F0417BF
:1069C800100540E02407340758F436F404910024F5
:1069D800F101E01BF0090994E00FF11F25903590B3
:1069E800F101099411F4D6F7F1CF31960EF03196F2
:1069F80050E060E070E045914B3F48F089F34F3F2D
:106A080029F04E3F11F07591659155914591041B00
:106A1800150B260B370B39F318F3E7CFFA92EA92E6
:106A2800DA92CA92BA92AA929A928A927A926A92BE
:106A38005A924A92BA93AA939A938A930895FF8492
:106A4800EE84DD84CC84BB84AA84998488847F8086
:106A58006E805D804C80BB81AA8199818881F0E03D
:106A6800EC0FFD1FEF0108950E941635229741E0B3
:106A780050E060E070E00E94A43460F440E00E94BE
:106A88009A3421F402E26BD03FEF5FC001E267D095
:106A98003FE75BC0AE010E94AB31C801D90143EFAB
:106AA80054E065E37FE30E94A43468F437FBAA0F3F
:106AB800BB1FB395B695A795B7F908811981015001
:106AC80010400883198340E050E060E87FEB43D032
:106AD8002801390140E050E060E87FE33CD0A8019C
:106AE800B901820193010E941B34C801D901A80190
:106AF800B9012FD0280139010881102F110F110B6E
:106B0800212F312F0E94E23248E152E761E37FE30F
:106B180020D04801590142E252E964ED7EE3820146
:106B2800930117D04DED5BE96AE27FE316D0A2012D
:106B3800B3010FD044E050E060E070E40ED0AC0147
:106B4800BD0107D0A401B50108D02296ECE00C9451
:106B580027350C94A2338C019D010C944133E8E94C
:106B6800F9E2008351830FEF1FEF2FE7089501E04B
:106B780008950E941235EF97EF976A972A873B8707
:106B88004887598768017B0100E00B830C8302C0AA
:106B980011D21BD20AD2053251F00023C9F70B815A
:106BA8001C81EF96EF966A96E0E10C9423350081FC
:106BB800053221F402D2FED105E2EBCF00E00F83CB
:106BC8000E830A8309833E0102E1600E00E0701E15
:106BD8000BE616E2088B198B06C00981002311F415
:106BE80000810983EAD1D9D10052B9F3035059F091
:106BF8000850B1F3025019F0035049F00CC00A8153
:106C080003950A83EFCF0E8103950E83EBCF0F8197
:106C180003950F83E7CF00810A3279F4AAD1AD90AA
:106C2800BD9098D1BB203AF4B194A19400E0B00A89
:106C38000A8103950A83C1D114C0AA24BB244AE05F
:106C480050E00DC021916F0185010E94E731A22E0D
:106C5800BB24A00EB11E00EDA00E0FEFB01EA0D1F8
:106C680088F30A81002311F000E00F8396D10E32D9
:106C7800F1F4A3D192D10A3231F47BD18D909D9059
:106C880069D19BD117C0882499244AE050E088D163
:106C980088F421916F0184010E94E731822E9924A2
:106CA800800E911E00ED800E0FEF901EF0CF88240D
:106CB8008A94982C80E071D10C5421F00C5131F059
:106CC800045039F481E0C80E7AD103C001E0C00E47
:106CD800D81E6BD1EEEAF3E00C94CD3480FB5EF461
:106CE8004B815C81652F660F660B47D140835183CA
:106CF800628363834FCF2B813C813FD120833183D3
:106D080049CF37D10D91119625D10A8B2E0103E178
:106D180015D1E0C02ED16D907D901CD1062D07298C
:106D280021F40CE7602E06E2702E992022F400E18F
:106D3800802E07E2902E80E090E001C00196F301DA
:106D480001913F01002319F088159905BCF30CD176
:106D58002301919581959040680E791EBBC00E81E4
:106D6800002331F0082D092919F4992488248394E3
:106D78000BE816E2088B198B0881003739F4F9D033
:106D8800ECD000E1D5D000E0098330C0F1D046F462
:106D98000D911D912D913D91DDD0C801D90101C002
:106DA800DCD008810F3611F408E0ECCF053749F73D
:106DB8000AE0E8CFDDD04D915D9126F46D917D918B
:106DC800C9D005C0C7D0652F660F660B762FCA01DC
:106DD800DB0177234AF40DE209839095A095B095DD
:106DE80081959F4FAF4FBF4F0AE0A2D03E0107E900
:106DF800600E00E0701E2E0107E9A0D0082F092BB5
:106E08000A2B0B2B11F001E001C000E00D83082DC7
:106E1800092919F40D8100FF1FC094D0E889F98968
:106E2800E00DF11D0081F30102933F018BD0C801F1
:106E3800D901012B022B032B81F799206AF40F81CA
:106E4800002351F0A3D010E04501801A910A04C034
:106E580000E3F30102933F018E0109561F4F061903
:106E6800170908151905A4F30E81002399F10D815E
:106E780000FF30C00881083711F0083549F474D094
:106E8800F3010881008370D000E3F301008322C07E
:106E98000F3601F5F30100810033E1F000E30293BE
:106EA8003F0118C00CE9602E06E2702E462C502EC9
:106EB800F2010081002371F001E040D0F9CF0FEF1B
:106EC800C00ED01E0FEB602E06E2702E02EC402E94
:106ED80006E2502E420186189708A814B9041CF43B
:106EE80080E090E007C052D0A818B90810E0A01AB6
:106EF800B10AC5010A81002321F401C063D00197BA
:106F0800EAF70981002339F055D004C053D0F301C2
:106F180001913F015AD00FEF800E901EBAF70A81F7
:106F2800002309F437CE01970AF434CE4BD0FBCFB7
:106F380010E00C871D871E871F870895400E00E00C
:106F4800501E08954C855D856E857F858C019D0159
:106F58000C945D32A083B18308958D919D91A08397
:106F6800B183A0E0B0E008950FEF600E701E0895A1
:106F780080FBF701A081B1810895F701A081B1815B
:106F88000D911D91A083B183F80108950981002313
:106F980011F001E0089500E00895F60100810895D8
:106FA800F601008100530A300895F60101916F013E
:106FB8000883089528853985089501E0C00E00E00A
:106FC800D01E08952885398500E2EA85FB85099554
:106FD8000B811C810F5F1F4F0B831C8308950E9438
:106FE8001E35C801D9011A013F7740E856E968E122
:106FF8007BE40E94BC3438F416D0B38300E010E080
:1070080020E030E00DC03B2F0E94EF320E94E232B8
:107018000AD03383A801B9018C019D010E948533F0
:10702800E4E00C942F35F101008311832283089545
:107038004DE65EE466EC71E4E3ECF6E20081118172
:10704800228133810E942D32075C1F4C2F4F3F4F06
:10705800008311832283338389011F7708950E9457
:107068001235C801D901BF7741E050E060E87FE3FD
:107078003B2F0E94A43470F440E00E949A3429F413
:107088000BED1FE029E43FE350C0CC24DD24EE24BF
:10709800FF241CC00BEDC02E0FE0D02E09E4E02E1B
:1070A800F72E40E07FEB082F48D02801390140E057
:1070B80050E060E87FE38C019D013FD0A801B90151
:1070C800820193010E941B34C801D901AC01BD01A2
:1070D8008C019D012DD02801390144E25FEF6BE25C
:1070E8007CEB26D048E854E466EA7EE328D048E101
:1070F80050EC6FE370E423D045EB1CD048015901F4
:107108004AEE54EB66E870E48201930118D046EB2E
:1071180011D0A801B901840195010E941B34AC016A
:10712800BD0106D0A601B70108D0E0E10C942335D3
:107138000C94A2335DEF68E670E40C944133FDDFF4
:10714800A201B301F5CF20E006D0E9F70895259113
:1071580002D0E9F708952D9301501040202F212BDC
:10716800089584E294E7FC0105911491FC0132969C
:10717800A591B491FC01349625913491422F432B6B
:1071880019F0F901E4DF01C0DEDF069614E7803369
:10719800910748F3089540E00C94D2380E941A35BC
:1071A8002897802FB32F442E40E050E060E070E035
:1071B8000E94A43410F401E001C000E0000F400E6A
:1071C800BF7743E859EF62E27FE3082F3B2F80D077
:1071D80076D041E05CEF6FE777E40E94BC3488F535
:1071E800AE010E94F3376BD0042D10E06BD04881BC
:1071F80059816A817B8172D0088319832A833B83F2
:10720800AE014C5F5F4F2A0140E050E060E87EE34A
:107218005FD0A2010E94F33740E050E060E870E4DC
:107228000C811D812E813F8153D0A801B9010881AD
:1072380019812A813B810E9485330E94EF32402EBA
:107248000CC00E94EF32602E3DD0A801B9018C011C
:107258009D0133D0460C03E0402240FA3EF4AC01D5
:10726800BD0100E010E020E83FE327D002E040162F
:1072780008F0B0588C019D0129D0280139014BEF45
:1072880057ED6EE179E324D045E656E269E97BEBF8
:1072980021D048E554E363EA7DE31CD041EE5DE587
:1072A80065E27FEB17D04BED5FE069EC7FE316D02A
:1072B8000DD02896E8E00C942B350E948533C80140
:1072C800D901089520E030E00C94ED32AC01BD0105
:1072D8000C94A23303D0A201B301FACF0C9441332A
:1072E8001B2F6A2FF901A081B181AD014F5F5F4F5C
:1072F800408351830C93A62FB12F0895BA93AA9374
:1073080024970A831B8389019E012A5F3F4F2883A4
:107318003983BE01AE014E5F5F4F24E739E30E9417
:10732800BD3520E0AA81BB812C932496A991B991FF
:1073380008950E94163522974801590141E050E00E
:1073480060E070E00E94A43498F440E00E949A340F
:1073580029F400E010E020E030E04EC001E2E8E966
:10736800F9E2008351830FEF1FEF2FE73FE744C097
:10737800AE010E94AB31C801D90145EC53E062E48B
:107388007FE30E9441334AE151E562E17FE33BD06C
:10739800A801B9018C019D013BD0402E088100FF56
:1073A80014C00A952DD0802F43EF54E065EB7FE39E
:1073B800042D0E94A23337FB220F331F380F369556
:1073C800279537F9C801D9010BC01AD0842D912F00
:1073D800D90137FBAA0FBB1FB00FB695A795B7F910
:1073E80040E050E060E87EE38C019D010CD0AC01E8
:1073F800BD01840195010CD02296ECE00C94273550
:1074080042E00C94D7310E94A23328013901089533
:107418000E941B34A201B3010C944133A30524211B
:107428003074D302C72600004E6F726D610046614A
:1074380073742000466173742B00466173742B2BA0
:107448000052415400564449004F4C4400416E6C70
:107458000042656C00412B53002D20504C45415390
:10746800452057414954202D20002020202020204D
:10747800203C3E20202020202020002021212120E7
:1074880053204F205320212121202000204C6F77AA
:107498002042617474657279202121210020202006
:1074A8003C20256420487A203E20202020002045CA
:1074B800524153494E4720454550524F4D212000D7
:1074C80050726F663D256420004B504F542D524139
:1074D80054494E472B207625642000203D20204427
:1074E8002045204D204F20203D202020002A2A2AF8
:1074F8002A20253032643A2530326420202A2A2A6C
:107508002A00466163746F72792073657474696EBA
:1075180067730020202053657474696E6773212097
:1075280020202000553D256420493D256420456DD7
:107538003D2564202020004D3D256420413D2564E3
:107548002047623D2564202A2564202000545820C5
:107558002564487A2025646D412020200052582057
:1075680025646D56202020200025645F25732000A7
:107578002020204572726F72204B3021002020207D
:107588005475726E20636F696C21002564762564DA
:10759800200020253032645F256400253032645F86
:1075A800256400203C202020202020202020203E70
:1075B80000203E202020202020202020203C003EAB
:1075C800232323232323232323233C005B2020205E
:1075D800202020205D002B253032645B205D202593
:1075E80064002D253032645B205D202564003C203A
:1075F8002020202F2020202020202020203E005B3B
:1076080020202020202050502020202020205D00F5
:1076180073257846256425630025642020202020D2
:10762800200050726F66696C652020202020202081
:1076380020200042617474657279202055623D25CE
:10764800642E256456005468726573682E20205491
:10765800623D25642E256456002B256420202020B9
:107668002D2E2E2E2E2E2E2E2E2B00436F6E747244
:107678002E20202020202020202020200025646D7E
:1076880041202020202020202020202020202000F1
:10769800282564292E2E2E20002A467265715F54F3
:1076A8005820256C64487A20002A466572726974ED
:1076B8006520200020202564256320200025303205
:1076C800643A2530326420436F64655F5F25303447
:1076D800582000456E742E5061732E3C303E202594
:1076E80030345820200025646D41202020200025BA
:1076F800632D2E2E2E2E2E2E2E2B00506F77657278
:107708002E20202020202020202020002A25642030
:1077180020202020202020002D2E2E2E2E2B200051
:107728004761696E20202020202020202020202052
:107738000025646D562020202020200020413D2572
:1077480064202020002A436F696C20626C2E20661A
:107758003D25642563202000464D20202020202040
:1077680020282D2920004F4646004F4E2000426C0D
:107778007565746F6F7468282B292000566F6C2EFE
:107788005B25635D2020202020202020202000254C
:10779800302E32643A25302E32645F25302E326422
:1077A80025634320534C45455020004D616E6C2E97
:1077B800663031323334353637382000253034647A
:1077C8003C202020202020202020203E00256474FA
:1077D8006F6E6520200025732D2E2E2E2E2B004235
:1077E8006565707320202020202020202020200084
:1077F8002573202020202020202020202020202029
:10780800004D6F646520202020202020202020208B
:1078180020003C25733E2020200053637265656E6E
:10782800202020202020202020200038363432300C
:107838002F3031323334353637385300436F6E7456
:10784800696E756520536574742E3F20004E6F2055
:10785800202020202020202020205965730020206F
:107868002020202020202020202020202020004709
:10787800726F756E6420626C2E4572726F72210091
:1078880047726F756E6420626C2E202D4F4B2D2031
:10789800002020202A2A2A202564202A2A2A20207B
:1078A80020200025302E32643A25302E32642020E4
:1078B80020202020200020202020202000202825F3
:1078C800303264293C253032643E20463D25642010
:1078D8000020204E6F204665727269746521202051
:1078E80020002054616B65204665727269746521B9
:1078F80020200020202020204572726F7221202035
:10790800202020002020202020204F4B2120202034
:1079180020202020002020202020206C6F6E67204F
:1079280020202020202000204F4B212000207261A1
:1079380064696F646F6D40692E7561202000202096
:107948002020204552524F52212020202020002064
:10795800202053657474696E6773202120202000ED
:10796800010AD7A3BC0AD7A3BC0AD7A3BC2C0130F1
:10797800313233343536373839414243444546008D
:10798800286E756C6C20706F696E74657229003092
:1079980031323334353637383961626364656600AD
:1079A800464C4F4154533F2077726F6E6720666F85
:1079B800726D617474657220696E7374616C6C6544
:0B79C8006421003F3F3F000100000071
:0400000300000000F9
:00000001FF
